:100000000C9473000C949B000C949B000C949B002C
:100010000C949B000C9460050C949B000C949B002A
:100020000C949B000C949B000C949B000C949B00E4
:100030000C949B000C949B000C949B000C949B00D4
:100040000C94E90C0C949B000C94D10B0C94AB0B0E
:100050000C949B000C949B000C949B000C949B00B4
:100060000C94860D0C949B001D141F142114231452
:100070002514271429142B145D14601463145A14C6
:10008000661469147A147A14000000002400270012
:100090002A0000000000250028002B0000000000BE
:1000A00023002600290004040404040404040202BA
:1000B00002020202030303030303010204081020E7
:1000C00040800102040810200102040810200000F2
:1000D0000008000201000003040700000000000007
:1000E00000000C2AB82911241FBECFEFD8E0DEBFD4
:1000F000CDBF26E0A6EEB3E001C01D92A336B20745
:10010000E1F713E0A0E0B1E0ECEAF5E602C005900B
:100110000D92A63EB107D9F710E0C2E7D0E004C0C7
:100120002197FE010E94092FC137D107C9F70E940C
:10013000DE1C0C94C9320C940000089580E090E01D
:100140000895CF93DF931F92CDB7DEB769832091D7
:10015000C3042223D1F02091E604203240F021E0B4
:1001600030E0FC013383228380E090E015C0809171
:10017000C404E82FF0E0EB53FB4F998190838F5F2D
:100180008093C4048093E60405C061E0CE0101962B
:100190000E94B40E81E090E00F90DF91CF9108951E
:1001A000CF92DF92EF92FF920F931F93CF93DF9343
:1001B000EB017B0124E0E20EF11C8B016C01C61AFD
:1001C000D70AC601800F911F0E941E2DF80181934E
:1001D0008F01EE15FF05A9F7CE01DF91CF911F9199
:1001E0000F91FF90EF90DF90CF900895AF92BF9264
:1001F000CF92DF92EF92FF920F931F93CF93DF93F3
:100200001F92CDB7DEB75C017B018B016C0184E0EE
:10021000C80ED11CF80161918F01C50169830E944C
:100220001E2D6981681719F0C5010E94262DFFEF68
:10023000AF1ABF0AAC14BD0469F7C7010F90DF9174
:10024000CF911F910F91FF90EF90DF90CF90BF90D3
:10025000AF900895CF93DF93EC0160E471E08AE002
:1002600090E00E94D000FC0180819181A281B38145
:100270008093400190934101A0934201B0934301C8
:100280006CE371E084E190E00E94D000FC01808189
:100290009181A281B38180933C0190933D01A09311
:1002A0003E01B0933F018091F0039091F1030097DC
:1002B00069F58091F503813009F46CC0C130D10536
:1002C00061F48091F6039091F703A091F803B09147
:1002D000F9030196A11DB11D10C0CF3FFFEFDF074D
:1002E00009F058C08091F6039091F703A091F803AC
:1002F000B091F9030197A109B1098093F603909396
:10030000F703A093F803B093F90344C0019709F0F1
:1003100041C0C130D105A9F4409140015091410143
:100320006091420170914301809144019091450197
:10033000A0914601B0914701840F951FA61FB71FDA
:1003400018C0CF3F2FEFD20711F580914001909157
:100350004101A0914201B09143014091440150916B
:1003600045016091460170914701841B950BA60BD6
:10037000B70B8093400190934101A0934201B09349
:10038000430160E471E08AE090E00E94F60081E0C1
:10039000809329048091F0039091F103029709F072
:1003A0004AC0C130D10539F580913C0190913D01A1
:1003B000A0913E01B0913F01805F984DAF4FBF4F7C
:1003C0008038E3EC9E07E9ECAE07E1E0BE0724F0DD
:1003D00080E893ECA9ECB1E080933C0190933D015F
:1003E000A0933E01B0933F016CE371E084E190E0A3
:1003F0000E94F6001DC0CF3FFFEFDF07C9F48091D8
:100400003C0190913D01A0913E01B0913F0180518E
:100410009742A109B109813026E392072EE6A2078F
:1004200021E0B207CCF680E096E3AEE6B1E0D4CFAF
:1004300081E0809329048091F0039091F103039768
:1004400009F04AC0C130D10539F5809190059091ED
:100450009105A0919205B0919305805C944BA34BBC
:10046000BF4F8115E9EE9E07E4EAAE07E5E3BE075C
:1004700024F080E099EEA4EAB5E380939005909390
:100480009105A0939205B093930560E975E08EE124
:1004900090E00E94F6001DC0CF3FFFEFDF07C9F4D8
:1004A0008091900590919105A0919205B09193054E
:1004B00080549B44AC44B109813026E4920723EC7C
:1004C000A20723E2B207CCF680E096E4A3ECB3E205
:1004D000D4CF81E0809329048091F0039091F103BF
:1004E0000497B1F58091F503813091F1C130D105C8
:1004F00039F580914C018F5F823008F082E0809363
:100500004C0180914C01813029F480E091EEA0E013
:10051000B0E006C0823061F480E092ECA1E0B0E08F
:100520008093380190933901A0933A01B0933B0135
:1005300068E371E088E290E0DF91CF910C94F600DF
:10054000219631F480914C018150C9F681E0D7CFDA
:10055000DF91CF910895CF93C1E087EE94E00E94A0
:10056000CA08181619062CF587EE94E00E94A80810
:100570008093E7030E94B81C8091E7038B3369F7EF
:10058000C093E60364E772E080EA95E00E94F80A0F
:1005900064E772E086E096E00E94F80A60E08FE08F
:1005A0000E945E1C64E273E083E596E00E94A90B62
:1005B000D4CFCF91089580E10E94030C892B61F480
:1005C0008091F303811108C08091F203811104C06E
:1005D00080912D04882329F080912C04813009F02A
:1005E0006EC081E08093EF0381E10E94030C892BB0
:1005F00059F480912A0490912B04892B29F480913D
:100600002904882309F45EC081E10E94030C01974C
:1006100039F480912A0490912B04019709F470C059
:100620008091F0039091F1030197E9F480912D04FA
:10063000811119C08091480190914901A0914A010E
:10064000B0914B018093230490932404A09325043C
:10065000B093260462EE75E08AEC95E00E940F0BE1
:1006600081E080932D0485E00E94030C019739F40A
:100670008091210490912204892B09F446C085E0E1
:100680000E94030C892B39F480912104909122045B
:10069000019709F44FC080911F04909120040097A6
:1006A00031F481E08093F3038093F203089501977E
:1006B00009F045C01092F3031092F20308951092CE
:1006C000EF0392CF81E090E020912704309128043D
:1006D000232B11F080E090E090932804809327046E
:1006E00081E090E090932B0480932A048091F003A2
:1006F0009091F10301969093F1038093F00384CFDE
:1007000010922B0410922A048BCF81E090E020916C
:100710001F0430912004232B11F080E090E090938F
:10072000200480931F0481E090E090932204809342
:100730002104A5CF1092220410922104ACCF089579
:100740008F929F92AF92BF92CF92DF92EF92FF92E1
:100750000F931F93CF93DF93CDB7DEB7AE970FB64E
:10076000F894DEBF0FBECDBF8091F0039091F103EE
:10077000019709F067C060E080E00E945E1C66E2BD
:1007800073E083E596E00E94A90B61E080E00E949F
:100790005E1C67E373E083E596E00E94A90B60911D
:1007A00040017091410180914201909143010E946A
:1007B0008E1C80E20E943A1B80E20E943A1B80E27B
:1007C0000E943A1B1092F5031092EF0310922C0432
:1007D00066E272E087EE94E00E94A90B6FE373E09B
:1007E00087EE94E00E94A90B66E470E080E090E060
:1007F0000E94AF0C6EE473E087EE94E00E94A90BB8
:1008000066E470E080E090E00E94AF0CA0904D01A3
:10081000B0904E01C0904F01D0905001E090510136
:10082000F09052010091530110915401812C912CB0
:1008300020E83BE346EE56E760E070E080E090E0C1
:100840000E9499168091F0039091F103029739F577
:1008500060E080E00E945E1C66E573E083E596E060
:100860000E94A90B61E080E00E945E1C62E872E0D9
:1008700083E596E00E94A90B60913C0170913D01D7
:1008800080913E0190913F010E948E1C67E673E0CB
:1008900083E596E00E94A90B80E20E943A1B8091BA
:1008A000F0039091F103039739F560E080E00E9436
:1008B0005E1C6BE673E083E596E00E94A90B61E0A5
:1008C00080E00E945E1C62E872E083E596E00E9490
:1008D000A90B60919005709191058091920590917E
:1008E00093050E948E1C62E872E083E596E00E9408
:1008F000A90B80E20E943A1B8091F0039091F103D2
:10090000049739F560E080E00E945E1C6CE773E0BC
:1009100083E596E00E94A90B61E080E00E945E1CE6
:1009200062E872E083E596E00E94A90B60913801CD
:100930007091390180913A0190913B010E948E1C87
:1009400062E872E083E596E00E94A90B80E20E94D3
:100950003A1B8091F0039091F10305970CF49DC030
:100960001092F1031092F00310922D046091230471
:100970007091240480912504909126041CA21BA24E
:100980001EA21DA218A61FA22AE0AE014F5F5F4F54
:100990000E948A2BBE016F5F7F4FCE0183960E941B
:1009A000F80A8FA198A50B9730F51AA619A61CA6D0
:1009B0001BA61EA61DA64AE0BE016F5F7F4F80E00A
:1009C00090E00E947F2BBE016F5F7F4FCE01899622
:1009D0000E94F80ABE016D5D7F4FCE0189960E948C
:1009E000C40ABC01CE0183960E940F0BCE018996EA
:1009F0000E94260BD6CF6BEB71E0CE0101960E94D0
:100A00002B0BBE016D5D7F4FCE0101960E94C40A83
:100A10000E94281BBC01CE0183960E940F0BCE01C1
:100A200001960E94260BBE016D5D7F4F87EE94E01C
:100A30000E94860B60E570E080E090E00E94AF0CC1
:100A40006DE873E0CE0101960E942B0B6AEC75E015
:100A5000CE0101960E94C40A0E94281BBC018AECA8
:100A600095E00E940F0BCE0101960E94260B6AECC6
:100A700075E087EE94E00E94860B60E570E080E010
:100A800090E00E94AF0C64E772E08AEC95E00E946F
:100A9000F80ACE0183960E94260BAE960FB6F89404
:100AA000DEBF0FBECDBFDF91CF911F910F91FF90A1
:100AB000EF90DF90CF90BF90AF909F908F90089570
:100AC0001F920F920FB60F9211242F933F934F93C3
:100AD0005F936F937F938F939F93AF93BF93CF93C6
:100AE000DF93EF93FF93809114060E94030CEC01B7
:100AF000809113060E94030CCC0FDD1F8C2BE0911C
:100B00001206EF7094E0E99FF0011124E80FF11D47
:100B1000E55AFE4F8081809312068073803119F46C
:100B20008FEF9FEF04C0803221F481E090E00E94BB
:100B30002A01FF91EF91DF91CF91BF91AF919F91EA
:100B40008F917F916F915F914F913F912F910F9076
:100B50000FBE0F901F9018951F93CF93DF9300D077
:100B600000D000D0CDB7DEB762E973E087EE94E045
:100B70000E94A90B87EE94E00E94480968E270E0A9
:100B800080E090E00E94AF0C87EE94E00E94CA08DB
:100B9000181619060CF052C087EE94E00E94A808BF
:100BA0008093E7038F3321F40E94AB020E94AC05CF
:100BB0008091E7038A3541F18091E6038823F1F1C2
:100BC00066E076E08CEA95E00E940F0B28E030E0CA
:100BD00045E050E06CEA75E0CE0101960E94400BC2
:100BE000BE016F5F7F4F86EA95E00E94790ACE01D1
:100BF00001960E94260B86EA95E00E94210A7093D6
:100C0000ED036093EC031AC08AE50E94B81C11E062
:100C100087EE94E00E94CA08181619066CF687EE53
:100C200094E00E94A8088093E7030E94B81C80917A
:100C3000E7038B3369F71093E603EACF64E772E0CA
:100C40008CEA95E00E94F80A64E772E086E096E09C
:100C50000E94F80A26960FB6F894DEBF0FBECDBFED
:100C6000DF91CF911F9108951F93CF93DF9300D011
:100C700000D000D0CDB7DEB769E973E087EE94E02D
:100C80000E94A90B87EE94E00E94480968E270E098
:100C900080E090E00E94AF0C87EE94E00E94CA08CA
:100CA000181619060CF07FC087EE94E00E94A80881
:100CB0008093E7038F3321F40E94AB020E94340635
:100CC0008091E7038A3531F08091E603882309F4A7
:100CD0006AC01AC08AE50E94B81C11E087EE94E051
:100CE0000E94CA08181619067CF787EE94E00E9445
:100CF000A8088093E7030E94B81C8091E7038B3318
:100D000069F71093E603EACF66E076E088EB95E0BA
:100D10000E940F0B25E030E044E050E068EB75E006
:100D2000CE0101960E94400BBE016F5F7F4F82EBA8
:100D300095E00E94790ACE0101960E94260B82EB73
:100D400095E00E94210A6093EE03611108C061E002
:100D500087E00E942C0C60E086E00E942C0C8091C1
:100D6000EE03813041F460E087E00E942C0C60E0EB
:100D700086E00E942C0C8091EE03823041F461E009
:100D800087E00E942C0C61E086E00E942C0C809190
:100D9000EE03833041F460E087E00E942C0C61E0B8
:100DA00086E00E942C0C64E772E088EB95E00E94DC
:100DB000F80A64E772E086E096E00E94F80A269658
:100DC0000FB6F894DEBF0FBECDBFDF91CF911F915C
:100DD00008950F931F93CF93DF938EE00E94980C9A
:100DE0008EE00E94980CEC016AE070E080E090E0F8
:100DF0000E94AF0C8EE00E94980C8EE00E94980C2E
:100E0000AC01990F660B770BCE010D2E000CAA0BCF
:100E1000BB0B8A019B010D5F1F4F2F4F3F4F0817E0
:100E200019072A073B076CF0435051096109710902
:100E300084179507A607B70724F0D0931E04C09324
:100E40001D04C0911D04D0911E04C53883E0D8074D
:100E500074F080912C04811105C010921C04109232
:100E6000290474C0813031F510921C046FC0CF3159
:100E7000D10504F580911C0481111CC0C0912C0483
:100E8000C1110AC061E084E00E942C0C81E08093D3
:100E90002C048093EF0381C0C13009F057C060E09B
:100EA00084E00E942C0C10922C041092EF03C0934B
:100EB0001C044CC0CE018197C99780F480911C041A
:100EC00081110AC067ED71E08CED95E00E942C0A5B
:100ED000882309F444C002C08130C1F1CE018B5592
:100EE0009109C49778F480911C04811109C06DE1C7
:100EF00072E08CED95E00E942C0A882399F102C0E3
:100F0000813021F1CE01805991098D9778F480913B
:100F10001C04811109C068EE71E08EEB95E00E941F
:100F20002C0A882351F102C0813081F0CE5BD109B7
:100F3000AB9760F480911C04811108C06BE073E0F2
:100F40008EEB95E00E942C0A8823D1F060E070E0DF
:100F5000CB01DF91CF911F910F910C94AF0C6FE9F2
:100F600073E002C065EA73E087EE94E00E94A90B8B
:100F700060EA70E080E090E00DC06BEA73E002C0D0
:100F80006FEA73E087EE94E00E94A90B64EB70E0D7
:100F900080E090E00E94AF0C81E080931C04D6CFEB
:100FA000CF930E94E90663EB73E087EE94E00E9422
:100FB000A90B87EE94E00E94480966E470E080E0A7
:100FC00090E00E94AF0C87EE94E00E94CA08892B43
:100FD00009F045C060E08DE00E942C0C0E94DB020D
:100FE0008091F4038F5F8093F40380911B048F5FE3
:100FF00080931B048091F0039091F103892B19F0E9
:101000000E94A003CECF60E080E00E945E1C67EBF0
:1010100073E083E596E00E94A90B8091F40386308B
:1010200061F461E080E00E945E1C68EC73E083E59F
:1010300096E00E94A90B1092F40380911B048C305F
:1010400009F0AFCF61E080E00E945E1C68EF72E0C3
:1010500083E596E00E94A90B10921B04A2CF61E0E9
:101060008DE00E942C0C87EE94E00E94CA081816AE
:1010700019068CF587EE94E00E94A8088093E70398
:101080008F3321F40E94AB020E94D0078091E703C6
:10109000893439F08091E6038823E9F01092E60361
:1010A0001AC089E40E94B81CC1E087EE94E00E9457
:1010B000CA081816190674F787EE94E00E94A8086B
:1010C0008093E7030E94B81C8091E7038B3369F794
:1010D000C093E603EACFCF9108950895CF92DF92AF
:1010E000EF92FF920F931F93CF93DF936C017A01DE
:1010F0008B01C0E0D0E0CE15DF0589F0D8016D91FD
:101100008D01D601ED91FC910190F081E02DC60199
:101110000995892B11F47E0102C02196ECCFC701FD
:10112000DF91CF911F910F91FF90EF90DF90CF90C3
:101130000895FC01538D448D252F30E0842F90E0DD
:10114000821B930B541710F0CF96089501970895C2
:10115000FC01918D828D981761F0828DDF01A80FBF
:10116000B11D5D968C91928D9F5F9F73928F90E0E1
:1011700008958FEF9FEF0895FC01918D828D981750
:1011800031F0828DE80FF11D858D90E008958FEF8D
:101190009FEF0895FC01918D228D892F90E0805C56
:1011A0009F4F821B91098F739927089587EE94E0D2
:1011B0000E94CA0821E0892B09F420E0822F0895BB
:1011C000FC01848DDF01A80FB11DA35ABF4F2C91E4
:1011D000848D90E001968F739927848FA689B789B3
:1011E0002C93A089B1898C9180648C93938D848D8C
:1011F000981306C00288F389E02D80818F7D80835B
:101200000895EF92FF920F931F93CF93DF93EC011A
:1012100081E0888F9B8D8C8D981305C0E889F989B2
:10122000808185FD24C0F62E0B8D10E00F5F1F4FCF
:101230000F731127E02E8C8DE8120CC00FB607FC3F
:10124000FACFE889F989808185FFF5CFCE010E9428
:10125000E008F1CF8B8DFE01E80FF11DE35AFF4F3F
:10126000F0820B8FEA89FB898081806207C0EE895A
:10127000FF896083E889F98980818064808381E0C7
:1012800090E0DF91CF911F910F91FF90EF90089523
:10129000CF93DF93EC01888D8823C9F0EA89FB891D
:1012A000808185FD05C0A889B9898C9186FD0FC014
:1012B0000FB607FCF5CF808185FFF2CFA889B989E9
:1012C0008C9185FFEDCFCE010E94E008E7CFDF9142
:1012D000CF91089580E090E0892B29F00E94D608F4
:1012E00081110C9400000895833081F028F481303E
:1012F00099F08230A1F008958730A9F08830B9F0D4
:101300008430D1F4809180008F7D03C08091800073
:101310008F7780938000089584B58F7702C084B55D
:101320008F7D84BD08958091B0008F7703C0809138
:10133000B0008F7D8093B00008953FB7F8948091FE
:10134000760490917704A0917804B091790426B541
:10135000A89B05C02F3F19F00196A11DB11D3FBFED
:10136000BA2FA92F982F8827820F911DA11DB11D7B
:10137000BC01CD0142E0660F771F881F991F4A9577
:10138000D1F7089585ED8093BC008091BC0084FD69
:10139000FCCF1092C20408950895E0917B048091DF
:1013A0007A04E81730F4F0E0E458FB4F808190E0D5
:1013B00008958FEF9FEF089590917B0480917A04B8
:1013C000981750F4E92FF0E0E458FB4F208130E00B
:1013D0009F5F90937B0402C02FEF3FEFC9010895F8
:1013E00080917A0490E020917B04821B91090895FA
:1013F0000E94AB320F931F93CF93DF93EC01888150
:101400009981009729F02A813B812617370788F4B4
:101410008B016F5F7F4F0E94E131009761F09983EC
:1014200088831B830A832C813D81232B11F4FC01CB
:10143000108281E001C080E0DF91CF911F910F9178
:101440000895FC0180819181009711F00C94582B34
:1014500060E070E0CB010895FC0124813581232BED
:1014600031F421E061157105A1F0FB0108C0FC0118
:10147000808191816115710531F421E0FC01808149
:10148000882339F005C00E94B93221E0892B09F088
:1014900020E0822F0895EF92FF920F931F93CF9336
:1014A000DF93FC01248135816115710511F480E021
:1014B00019C041155105A9F07B01EC018A01020F09
:1014C000131FB8010E94FA09882389F32881398102
:1014D0008C819D81B701820F931F0E94C2321D83B0
:1014E0000C8381E0DF91CF911F910F91FF90EF90DE
:1014F00008950F931F93CF93DF938C01EB01FC01B1
:10150000808191810097B1F06881798161157105C1
:1015100079F0428153812C813D814217530740F07D
:101520000E94C2328C819D81F8019583848313C00F
:101530000E94493188819981F801918380838A8151
:101540009B81938382838C819D819583848319827F
:1015500018821B821A821D821C82DF91CF911F91FB
:101560000F910895CF93DF93EC01888199810097C3
:1015700011F00E944931198218821D821C821B823F
:101580001A82DF91CF910895CF93DF93EC01FB0195
:1015900044815581608171810E944B0A811103C091
:1015A000CE010E94B20ACE01DF91CF910895EF9251
:1015B000FF920F931F93CF93DF93EC017B018A017E
:1015C000BA010E94FA09811104C0CE010E94B20A38
:1015D00007C01D830C83B701888199810E94C232A4
:1015E000CE01DF91CF911F910F91FF90EF90089561
:1015F000CF93DF93EC016115710559F0FB01019068
:101600000020E9F73197AF01461B570B0E94D70A1C
:1016100002C00E94B20ACE01DF91CF910895CF930C
:10162000DF93EC01FB018617970761F06081718100
:101630006115710529F0448155810E94D70A02C0C5
:101640000E94B20ACE01DF91CF910895FC01808102
:1016500091810C944931FC01118210821382128213
:10166000158214826115710551F0FB010190002073
:10167000E9F73197AF01461B570B0C94D70A089531
:10168000BF92CF92DF92EF92FF920F931F93CF936F
:10169000DF937C016B018A01E9012417350720F4EF
:1016A000812F8901C42FD82F64E772E0C7010E94FF
:1016B0002B0BD60114968D919C911597081719073D
:1016C000D0F48C179D0708F4EC01D601ED91FC9144
:1016D0001197EC0FFD1FB08010824D915C91BA0103
:1016E000600F711FC7010E94F80AD601ED91FC91AD
:1016F000EC0FFD1FB082C701DF91CF911F910F91B9
:10170000FF90EF90DF90CF90BF900895DC01ED91B6
:10171000FC91DB0114964D915C9115976D917C9134
:101720000280F381E02D09946115710579F0FB01C8
:1017300001900020E9F73197AF01461B570BDC0100
:10174000ED91FC910280F381E02D099480E090E01E
:1017500008950C94940B1F920F920FB60F921124C0
:101760002F933F934F935F936F937F938F939F93A9
:10177000AF93BF93EF93FF9387EE94E00E94E0084E
:10178000FF91EF91BF91AF919F918F917F916F9159
:101790005F914F913F912F910F900FBE0F901F902F
:1017A00018951F920F920FB60F9211242F938F93BB
:1017B0009F93EF93FF93E091F704F091F8048081F9
:1017C000E091FD04F091FE0482FD12C090818091B1
:1017D00000058F5F8F7320910105821751F0E09112
:1017E0000005F0E0E951FB4F958F8093000501C0A3
:1017F0008081FF91EF919F918F912F910F900FBE5C
:101800000F901F901895CF93DF93282F30E0F901A8
:10181000E253FF4F8491F901E654FF4FD491F9014F
:10182000EA55FF4FC491CC2391F081110E947409B5
:10183000EC2FF0E0EE0FFF1FE456FF4FA591B4919F
:10184000EC91ED2381E090E021F480E002C080E0A3
:1018500090E0DF91CF9108951F93CF93DF93282FCE
:1018600030E0F901E253FF4F8491F901E654FF4F54
:10187000D491F901EA55FF4FC491CC23C9F0162F3A
:1018800081110E947409EC2FF0E0EE0FFF1FEE565D
:10189000FF4FA591B4918FB7F894111105C09C9199
:1018A000ED2FE095E92302C0EC91ED2BEC938FBF77
:1018B000DF91CF911F910895CF93DF9390E0FC01CA
:1018C000E654FF4F2491FC01EA55FF4F8491882391
:1018D00061F190E0880F991FFC01E857FF4FC59117
:1018E000D491FC01EE56FF4FA591B491611109C04E
:1018F0009FB7F8948881209582238883EC912E23CA
:101900000BC0623061F49FB7F8943881822F8095C4
:1019100083238883EC912E2B2C939FBF06C08FB717
:10192000F894E8812E2B28838FBFDF91CF91089503
:101930008E3008F08E508770806480937C00809198
:101940007A00806480937A0080917A0086FDFCCFD3
:10195000809178002091790090E0922B08958F92E9
:101960009F92AF92BF92CF92DF92EF92FF926B0164
:101970007C010E949D094B015C01C114D104E1046A
:10198000F104F1F00E949D09DC01CB01881999094D
:10199000AA09BB09883E9340A105B10570F321E077
:1019A000C21AD108E108F10888EE880E83E0981E7B
:1019B000A11CB11CC114D104E104F10419F7DDCF5D
:1019C000FF90EF90DF90CF90BF90AF909F908F905F
:1019D00008951F920F920FB60F9211242F933F93E9
:1019E0008F939F93AF93BF938091E8039091E90306
:1019F000A091EA03B091EB033091750423E0230F2B
:101A00002D3720F40196A11DB11D05C026E8230F36
:101A10000296A11DB11D209375048093E803909355
:101A2000E903A093EA03B093EB03809176049091CD
:101A30007704A0917804B09179040196A11DB11D9D
:101A40008093760490937704A0937804B0937904FC
:101A5000BF91AF919F918F913F912F910F900FBEAA
:101A60000F901F901895FC01248131E03093C3043E
:101A70002093E5041092C4041092E6048385682B39
:101A800084E895E00E94A1000C947B120F931F93B1
:101A9000CF938C01C62F0E94330D6C2F6460C80158
:101AA0000E94330D6C2F6B7FC8010E94330D83ECB5
:101AB00090E00197F1F7CF911F910F910895FF9258
:101AC0000F931F93CF93DF931F92CDB7DEB78C0197
:101AD000F62E962F907F692F642BC80149830E94B0
:101AE000460D80E1F89EB00111244981642BC801A4
:101AF0000F90DF91CF911F910F91FF900C94460DA5
:101B000041E00E945F0D81E090E008951F920F92E6
:101B10000FB60F9211242F933F934F935F936F93C0
:101B20007F938F939F93AF93BF93EF93FF93809196
:101B3000B900887F803609F49CC068F5883209F4C2
:101B40005BC090F4803109F454C038F4882309F460
:101B5000F6C0883009F44DC0F6C0883109F44CC095
:101B6000803209F45DC0EFC0803409F468C048F4E5
:101B7000803309F455C0883309F0E5C08093C00470
:101B8000D8C0803509F44FC0883509F45DC0883469
:101B900009F0D9C0D6C0883909F4C7C0A8F488377D
:101BA00009F467C038F4883609F463C0803709F453
:101BB00060C0C9C0883809F4B8C0803909F45FC072
:101BC000803809F0C0C05BC0803B09F486C038F49F
:101BD000803A09F466C0883A09F47FC0B4C0803CFA
:101BE00009F4A7C0883C09F4A4C0883B09F48AC062
:101BF000AAC080919D0410C09091BF048091BE0442
:101C0000981770F5E091BF0481E08E0F8093BF04B8
:101C1000F0E0E256FB4F80818093BB0085EC86C0EC
:101C20008093C0048EC0E091BF0481E08E0F80934A
:101C3000BF048091BB00F0E0E256FB4F808390919F
:101C4000BF048091BE046EC0E091BF0481E08E0F9E
:101C50008093BF048091BB00F0E0E256FB4F80838D
:101C60008091C10481116DC081E080939C0484EA5D
:101C700061C083E08093C20410927404CFCF80913E
:101C80007404803208F051C0E091740481E08E0F3A
:101C9000809374048091BB00F0E0EC5AFB4F80838A
:101CA000BDCF85EC8093BC001092C2048091740477
:101CB000803230F4E0917404F0E0EC5AFB4F108273
:101CC0006091740470E0E0915204F091530484E553
:101CD00094E009951092740436C084E08093C204A5
:101CE0001092510410925004E0914E04F0914F0470
:101CF000099580915004811105C081E080935004C2
:101D000010922E04E091510481E08E0F80935104D3
:101D1000F0E0E25DFB4F80818093BB009091510425
:101D200080915004981708F479CF85E88093BC001F
:101D30000AC085EC8093BC001092C20404C01092CB
:101D4000C0040E94C209FF91EF91BF91AF919F9192
:101D50008F917F916F915F914F913F912F910F9054
:101D60000FBE0F901F90189540915004262F30E021
:101D7000240F311D21323105DCF42091C2042430BE
:101D8000C9F4FC0180E090E0861758F430915004CB
:101D90002191DC01A25DBB4FA30FB11D2C930196D5
:101DA000F3CF80915004680F6093500480E0089551
:101DB00081E0089582E00895CF92DF92EF92FF9242
:101DC0000F931F93CF93DF937C01262F972F8A01C8
:101DD0008091C304882391F0C62FD72F6E01C40EC3
:101DE000D51ECC15DD0571F06991D701ED91FC91FF
:101DF0000190F081E02DC7010995F3CF642F822F68
:101E00000E94B40EC801DF91CF911F910F91FF90F6
:101E1000EF90DF90CF9008951092C20481E08093FC
:101E2000C10410929C0461E082E10E942C0C61E0EC
:101E300083E10E942C0CE9EBF0E080818E7F8083AF
:101E400080818D7F808388E48093B80085E48093CF
:101E5000BC0008952F923F924F925F926F927F92B3
:101E60008F929F92AF92BF92CF92DF92EF92FF92AA
:101E70000F931F93CF93DF93CDB7DEB76A970FB65B
:101E8000F894DEBF0FBECDBF322E232E4D875E8766
:101E90003B012C01A982B98ACA8ADB8AEC8AFD8AB5
:101EA0000E8B1F8B988A8F86211500EA30070CEA6B
:101EB000400709EB500703E06007710581059105B4
:101EC00011F008F046C02F3F10EE310715EF410723
:101ED00015E05107610571058105910561F058F024
:101EE0002F3F354D41415E476340710581059105A6
:101EF00009F0D8F50BC0312CB1EE2B2EF5EFFD8794
:101F000005E00E87612C712C412C512C29813989D7
:101F10004A895B896C897D898E899F89A0E00E94AE
:101F2000943009F0AEC0A32CB22CCD84DE847301B2
:101F3000820120E034E04BE654EF64E170E080E0A1
:101F400090E00E94D52F29873A874B875C87912C98
:101F500024C0312CF0EA2F2E1CEA1D8729EB2E8796
:101F6000A3E06A2E712C412C512C298139894A8990
:101F70005B896C897D898E899F89A0E00E9494305D
:101F800009F025C19924939414E0E12EF12C00E08E
:101F900010E0E986FA860B871C87E984FA840B85B2
:101FA0001C85A801970160E070E0CB01A32CB22C46
:101FB000CD84DE847301820129833A834B835C8361
:101FC0006D837E838F83988760E070E080E090E08F
:101FD0000E940F2F2983398B4A8B5B8B6C8B7D8BF7
:101FE0008E8B9F8BFF24F3949F1409F4F3C010E0B1
:101FF000812C912C54018394C12CD12C760101C0E9
:1020000011E007E0CC0CDD1CEE1CFF1C0A95D1F79B
:10201000C701B601A50194010E94C82E89859A8541
:10202000AB85BC8567E0880F991FAA1FBB1F6A9507
:10203000D1F79250A109B109820F931FA41FB51FB8
:10204000EF85F88980839183A283B383C501B401AE
:102050000E94A42EC61AD70AE80AF90AC482D582B9
:10206000E682F78280869186A286B3861111E5C04A
:10207000298139894A895B896C897D898E899F8903
:10208000E2C01A8EA32CB22CCD84DE8473018201AF
:10209000298139894A895B896C897D898E899F89E3
:1020A0000E94D52F29873A874B875C8789859A8537
:1020B000AB85BC850697A105B10520F4F6E0AF2EEF
:1020C000B12C0FC0E984FA840B851C8529E0E21647
:1020D00027E0F20601051105D0F078E0A72EE7E031
:1020E000BE2EC12CD12CE12CF12C00E010E0298176
:1020F00039894A895B896C897D898E899F890E948B
:10210000D52F322E232E4D875E873B012C01A32C29
:10211000B22CCD84DE8473018201298139894A89F8
:102120005B896C897D898E899F890E94D32F4901A3
:10213000B42FA52FF62FE72F888F998F05E00E94E7
:1021400042305401CB2EDA2EEF2EFE2E088D198D43
:102150000E94823005E00E944230088D0E94793052
:1021600005E00E944230088D0E948230288F398F0E
:102170004A01B62FA72FF82FE92F6B2F7A2F8F2F19
:102180009E2F05E00E94423059016A017B018C01BB
:10219000288D398DA4016B2F7A2F8F2F9E2F0E94AF
:1021A0007930A32CB22CCD84DE84730182010E948D
:1021B000D52FC22ED32EE42EF52EC114D104E10466
:1021C000F104F9F4812C912C5401839420C081E016
:1021D0008A8F58CFAF85B8891D921D921D921C928F
:1021E0001397FD011482158216821782C12CD12CFF
:1021F0007601C3941896CD92DD92ED92FC921B97D6
:1022000022C088248A94982C8FE0A82EB12CFA8DB5
:10221000F13009F0F5CEEF85F88910821182128233
:102220001382148215821682178281E090E0A0E06A
:10223000B0E080879187A287B387232D322D4D850B
:102240005E85B301C2016A960FB6F894DEBF0FBE79
:10225000CDBFDF91CF911F910F91FF90EF90DF9055
:10226000CF90BF90AF909F908F907F906F905F9036
:102270004F903F902F900895DF92EF92FF920F932F
:102280001F93CF93DF93FC01E080F18002811381E3
:10229000D481C581B681D7809701A8016D2F7C2F8D
:1022A0008B2F9D2D35534C405109610971098109CE
:1022B00091092F3F34434C4051056105710581055B
:1022C000910509F098F49701A8016D2F7C2F8B2FB1
:1022D0009D2D07E00E944230208331834283538347
:1022E000648375838683978387E0FDC09701A80187
:1022F0006D2F7C2F8B2F9D2D3A5648415109610936
:102300007109810991092F3F3946484151056105FD
:1023100071058105910509F098F49701A8016D2FC9
:102320007C2F8B2F9D2D06E00E944230208331832D
:1023300042835383648375838683978386E0D3C007
:102340009701A8016D2F7C2F8B2F9D2D345D40436D
:10235000510961097109810991092F3F334D4043AA
:102360005105610571058105910509F098F4970102
:10237000A8016D2F7C2F8B2F9D2D05E00E944230F0
:102380002083318342835383648375838683978359
:1023900085E0A9C09701A8016D2F7C2F8B2F9D2D63
:1023A000385A4146510961097109810991092F3F44
:1023B000374A41465105610571058105910509F0CE
:1023C00098F49701A8016D2F7C2F8B2F9D2D04E091
:1023D0000E94423020833183428353836483758318
:1023E0008683978384E07FC09701A8016D2F7C2F9F
:1023F0008B2F9D2D3055434C51096109710981097D
:1024000091092F3F3F44434C5105610571058105FA
:10241000910509F098F49701A8016D2F7C2F8B2F5F
:102420009D2D03E00E9442302083318342835383F9
:10243000648375838683978383E055C09701A801E1
:102440006D2F7C2F8B2F9D2D305A464851406109AE
:102450007109810991092F3F3F4946485140610563
:1024600071058105910509F098F49701A8016D2F78
:102470007C2F8B2F9D2D02E00E94423020833183E0
:1024800042835383648375838683978382E02BC062
:102490009701A8016D2F7C2F8B2F9D2D30544D401F
:1024A000534061097109810991092F3F3F434D4014
:1024B0005340610571058105910509F098F4970174
:1024C000A8016D2F7C2F8B2F9D2D01E00E944230A3
:1024D0002083318342835383648375838683978308
:1024E00081E001C080E0DF91CF911F910F91FF90BB
:1024F000EF90DF9008952091E6049091E504213259
:1025000008F04AC08091C2048111FCCF32E03093C0
:10251000C20431E03093C1043FEF3093C004109205
:10252000BF042093BE04A5ECB4E04EE954E0FA01E8
:102530003E2F341B321718F43D913193F9CF10928E
:102540009D0420919D04990F922B90939D0490914E
:102550009C04913061F410929C0490919D0490939E
:10256000BB009091BC0093FDF8CF95EC01C095EEB7
:102570009093BC009091C2049230E1F39091C0041A
:102580009F3F79F08091C004803241F08091C00477
:10259000803331F084E005C081E003C082E001C0F7
:1025A00083E01092C4041092E6041092C3040895CC
:1025B000EF92FF920F931F93CF93DF931F92CDB7AC
:1025C000DEB7162F91E09093C30490E69093E50454
:1025D0001092C4041092E604682F84E895E0798391
:1025E0000E94A100E12E7981F72E8701085F1F4F1D
:1025F000F70161917F0184E895E00E94A100E01657
:10260000F106B1F70F90DF91CF911F910F91FF90DD
:10261000EF900C947B12EF92FF920F931F93CF9346
:10262000DF931F92CDB7DEB7162F877028E0829F09
:10263000C0011124682F606440E083E596E079834F
:102640000E945F0DE12E7981F72E8701085F1F4FF1
:10265000F70161917F0183E596E00E94800DE0160D
:10266000F106B1F70F90DF91CF911F910F91FF907D
:10267000EF900895CF93C62F91E09093C30490E616
:102680009093E5041092C4041092E604682F84E845
:1026900095E00E94A1006C2F84E895E00E94A100C3
:1026A000CF910C947B12CF93DF9391E09093C3046E
:1026B00090E69093E5041092C4041092E604682F0B
:1026C00084E895E00E94A1000E947B128091C204E0
:1026D0008111FCCF91E09093C2041092C1048FEF5E
:1026E0008093C0041092BF041092BE0490939D0486
:1026F00090919D04906C90939D0480919C048130F6
:1027000061F410929C0480919D048093BB008091A1
:10271000BC0083FDF8CF85EC01C085EE8093BC0042
:102720008091C2048130E1F38091BF04811103C024
:10273000C091BF0401C0C1E0AEE9B4E02CE734E0D1
:10274000F9018E2F821B8C1718F48D918193F9CF8C
:1027500010927B04C0937A0480917B04C81731F0F7
:1027600084E895E00E94DC09D82FF6CF8D2FDF9109
:10277000CF9108952F923F924F925F926F927F92E6
:102780008F929F92AF92BF92CF92DF92EF92FF9281
:102790000F931F93CF93DF93CDB7DEB72E970FB66E
:1027A000F894DEBF0FBECDBF982E792E49875A8789
:1027B0006B877C876BA05C2C2D2C3E2D402E312E00
:1027C000C984DA84EB84FC8484E190E02E873D8721
:1027D0000E94B4308C01FC01D082C182892D880F07
:1027E000880F880F845D0E9453138C7F3D85932F43
:1027F0009370892BF801828323825482D701C6010A
:102800006CE0B695A795979587956A95D1F7982F1F
:10281000907F2E85822F8F70C82EC90EC58236827A
:102820004782E92CF72CF8E0EF16F104B8F4F70131
:10283000EC5CFF4FB8010C94092F8AE20DC082E3D3
:102840000BC08AE309C082E407C08AE405C082E5C0
:1028500003C08AE501C08BE50E94D81280E1980E82
:10286000892D0E94531391E0682FA91202C0606461
:1028700001C06F7B892D0E943A13E1E0EE16F1044E
:1028800051F0F2E0EF16F10449F0E114F10449F4DB
:10289000A092460612C0A092470612C0A092480617
:1028A00012C088E0E816F104B0F4F701E45CFF4FD1
:1028B0000C94092F54E4B52E0EC04CE2B42E0BC07C
:1028C00034E3B32E08C02CE3B22E05C09CE4B92E2D
:1028D00002C084E5B82E8B2D0E94531383786110BB
:1028E0008C6090E1899E40011124682F68298B2D0E
:1028F0000E943A13C8012E960FB6F894DEBF0FBEA1
:10290000CDBFDF91CF911F910F91FF90EF90DF909E
:10291000CF90BF90AF909F908F907F906F905F907F
:102920004F903F902F900C9449310F931F93CF936A
:102930008B01C0E1C80F8C2F0E94531301151105A4
:1029400011F48F7D04C00130110509F48062682FF5
:102950008C2FCF911F910F910C943A132F923F928D
:102960004F925F926F927F928F929F92AF92BF929F
:10297000CF92DF92EF92FF920F931F93CF93DF934B
:10298000CDB7DEB763970FB6F894DEBF0FBECDBFED
:10299000322E3A874B875C876D87272E2C011F8745
:1029A0000E8760914F06709150068091510690916C
:1029B000520624E630E040E050E00E94772F2A8B58
:1029C0003B8B4D835E83762E672E888B998B80910F
:1029D000490690914A06A0914B06B0914C066C01B5
:1029E0007D01FF0CCC08DC2C76019C01AD016C2D27
:1029F0007C2D8C2D9C2D0FE10E944230A12CEAEC05
:102A0000BE2EFAE9CF2EABE3DA2EE12CF12C00E05A
:102A100010E00E94A42FAA88BB88CD80DE80E72C1E
:102A2000F62C088919890E940F2F0FE10E945D3052
:102A300049015A01D501C401BB0F880B982FDC0155
:102A400089839A83AB83BC839401A5016981762F26
:102A5000862F962FAA88BB88CD80DE80E72CF62CA7
:102A600008890E94793039014A01698B788B898302
:102A70009D83232D3A854B855C856D85722DC20122
:102A80002F3FA7E53A07A7E44A07A8EF5A07ADE0AA
:102A90006A07710581059105A9F0A0F02115344060
:102AA0004B46544F6441710581059105B9F0B0F072
:102AB000312CA4E0AA87BBE6BB87E4EFEC87F4E106
:102AC000FD8709C0312CE8E5EA87F7E4FB8788EF4A
:102AD0008C879DE09D87212C412C512C5301640152
:102AE000E988F88809811D81232D3A854B855C850D
:102AF0006D85722DC2010E94D52F2E833F8348879A
:102B000059878E819F81A885B9850F97A105B10549
:102B100058F49301A401B701C80104E00E944230B7
:102B200009810E94823028C08E819F81A885B98545
:102B30008B359105A105B10530F19301A401698997
:102B4000788989819D8102E00E94423053016401AD
:102B5000E988F88809811D810E94823059016A0143
:102B60007B01E82F192F04E00E9442300E2F0E94B3
:102B7000823001E00E944230322E3A874B875C87D8
:102B80006D87272E2C0153016401E988F88809819B
:102B90001D81232D3A854B855C856D85722DC20183
:102BA0000E94D32F2901B42FA52FF62FE72F382EFF
:102BB000292E05E00E9442305201CB2EDA2EEF2E54
:102BC000FE2E032D122D0E94823005E00E9442301D
:102BD000032D0E94793005E00E944230032D0E94AF
:102BE000823019012A01B62FA72FF82FE92F05E00F
:102BF0000E94423059016A017B018C019101A201BE
:102C00006B2F7A2F8F2F9E2F0E94793053016401F2
:102C1000E988F88809811D810E94D52F69017A0110
:102C2000C114D104E104F10429F4812C912C540144
:102C3000839406C088248A94982C3FE0A32EB12C5C
:102C400087E0CC0CDD1CEE1CFF1C8A95D1F7C70178
:102C5000B601A50194010E94C82E4E805F80688451
:102C6000798497E0440C551C661C771C9A95D1F723
:102C700092E0591A61087108420E531E641E751EB7
:102C8000C501B4010E94A42EC61AD70AE80AF90A9F
:102C900084E190E00E94B4308C01DC019C9211969A
:102CA0008C921197862D837012968C93129713969F
:102CB0005C92139714964C92D501C4012CE0B69502
:102CC000A795979587952A95D1F7982F907F8E2D68
:102CD0008F70882E890EF8018582D682C7828E85F4
:102CE0009F85892B19F4B8018AE106C0AE85BF859E
:102CF000119721F4B80182E20E94D812C8016396AC
:102D00000FB6F894DEBF0FBECDBFDF91CF911F91FC
:102D10000F91FF90EF90DF90CF90BF90AF909F907A
:102D20008F907F906F905F904F903F902F900C947A
:102D300049312F923F924F925F926F927F928F9282
:102D40009F92AF92BF92CF92DF92EF92FF920F933A
:102D50001F93CF93DF93CDB7DEB7AB970FB6F89441
:102D6000DEBF0FBECDBF298F3A8F4B8F5C8F6D8F2B
:102D70007E8F8F8F98A37A2CB9A2CAA2DBA23E2C99
:102D80004F2C602E212E9AA689A62A2D3B2DA60116
:102D90006E2D7F2D802F912FA0E00E94943091F016
:102DA00038554744584F6D407109810991092115E3
:102DB0003C4A43425C4F664071058105910511F024
:102DC00008F028C4298D3A8D4B8D5C8D6D8D7E8DDC
:102DD0008F8D98A12F3F34434C40510561057105FB
:102DE0008105910509F050F4198E85E38A8F8CE0F6
:102DF0008B8F1C8E1D8E1E8E1F8E18A2298D3A8DD4
:102E00004B8D5C8D6D8D7E8D8F8D98A12115304AF7
:102E10004C4A594B634071058105910569F060F09A
:102E2000198E80EA8A8F8CEA8B8F89EB8C8F83E0F6
:102E30008D8F1E8E1F8E18A2CE0149960E943C11C6
:102E40008BA7272D39A14AA15BA1632D742D862D57
:102E5000922DA0E0B98DFA8DEB8D0E94943009F48B
:102E600083C0AC8D8D8D5E8C9F8D9EA318A118A7FD
:102E70002B2F3F2F4E2F5A2F682F752D892F912FD3
:102E80002F3F15ED310711E141071EE7510713E010
:102E9000610771058105910511F008F065C0CE014B
:102EA0000D964C01A72CB9A0CAA0DBA0E32CF42CF2
:102EB000062D122D8EA198A50E942A0F89A59AA5EC
:102EC00081309105F9F082309105A9F1892B09F043
:102ED0007AC3898D80932E068A8D80932F068B8DE1
:102EE000809330068C8D809331068D8D80933206D1
:102EF0008E8D809333068F8D8093340688A18093C6
:102F0000350661C3898D809336068A8D8093370696
:102F10008B8D809338068C8D809339068D8D8093B0
:102F20003A068E8D80933B068F8D80933C0688A158
:102F300080933D0648C3898D80933E068A8D809399
:102F40003F068B8D809340068C8D809341068D8D3E
:102F5000809342068E8D809343068F8D8093440626
:102F600088A1809345062FC39C8D1D8D1CA35E8C6C
:102F70008F8D8EA3A8A12B2F3F2F4E2F592F612F5E
:102F8000752D9A2F2F3F15ED310711E141071EE7EF
:102F9000510713E06107710581059105D9F0D0F063
:102FA000CE010D964C01A12CB12CC12CD12CE12CC1
:102FB000F12C00E010E08EA19A2F0E942A0F722EB1
:102FC00039A34AA35BA3362E472E682E292E91E003
:102FD0009FA301C01FA289A59AA58130910509F47C
:102FE0005AC08230910509F4A0C1892B09F012C39F
:102FF000298D3A8D4B8D5C8D6D8D7E8DCE010D961C
:103000004C01A12CB12CC12CD12CE12CF12C00E0D5
:1030100010E08F8D98A10E942A0F722E39A34AA327
:103020005BA3362E472E682E292E60E070E080E0EC
:1030300090E00E94951470921E0699A190931F062D
:10304000EAA1E09320061BA11093210630922206EC
:10305000409223066092240620922506898D809353
:103060002E068A8D80932F068B8D809330068C8D53
:10307000809331068D8D809332068E8D809333063A
:103080008F8D8093340688A1809335065524539400
:103090001DA21CA29AC280914E06E98DECA3EA8D76
:1030A000EEA3EB8DE8A75C8CBD8DAE8DFF8DE8A106
:1030B000823009F075C02CA13EA148A5552D6B2F7B
:1030C0007A2F8F2F9E2F30584A415640610971093F
:1030D000810991092F37304E4247584962407105A6
:1030E0008105910569F160F1A0903E06B0903F0620
:1030F000C0904006D0904106E0904206F090430612
:1031000000914406109145062CA13EA148A5552DDD
:103110006B2F7A2F8F2F9E2F0E948B3089F0109269
:103120003606109237061092380610923906109221
:103130003A0610923B0610923C0610923D066AC277
:10314000709026068091270689A3909128069AA35D
:10315000109129061BA330902A0640902B06609000
:103160002C0620902D06CE010D964C01A72CB9A05F
:10317000CAA0D12EE32CF42C062D122D2CA13EA199
:1031800048A5552D6B2F7A2F8F2F9E2F0E942A0F27
:1031900061E070E081E090E00E949514512C38C00D
:1031A0007092260699A1909327061AA110932806DB
:1031B0008BA18093290630922A0640922B066092BA
:1031C0002C0620922D06CE010D964C01A12CB12C7F
:1031D000C12CD12CE12CF12C00E010E02CA13EA15F
:1031E00048A5552D6B2F7A2F8F2F9E2F0E942A0FC7
:1031F000722E39A34AA35BA3362E472E682E292EA2
:1032000061E070E081E090E00E94951455245394B1
:10321000298D3A8D4B8D5C8D6D8D7E8D8F8D98A116
:1032200030584A41564061097109810991092F3787
:10323000304E42475849624071058105910509F0B9
:1032400008F457C081E080934E0620913E063091ED
:103250003F064091400650914106609142067091B0
:1032600043068091440690914506A0E00E94943068
:1032700009F442C08EE396E00E943C118BA7A09017
:103280002606B0902706C0902806D0902906E09028
:103290002A06F0902B0600912C0610912D06209105
:1032A0003E0630913F0640914006509141066091A4
:1032B000420670914306CE0101964C01809144066E
:1032C000909145060E942A0F1F928BA4A12CC980C1
:1032D000DA80EB80FC800D811E812F813885498545
:1032E0005A856B857C8582E090E00E94BA130F902E
:1032F00003C088E080934E06898D809336068A8DC0
:10330000809337068B8D809338068C8D8093390699
:103310008D8D80933A068E8D80933B068F8D8093A2
:103320003C0688A180933D0649C190904E06E98DE8
:10333000ECA3EA8DEEA3EB8DE8A75C8CBD8DAE8D82
:10334000FF8DE8A111E0911275C02CA13EA148A506
:10335000552D6B2F7A2F8F2F9E2F30584A41564074
:1033600061097109810991092F37304E4247584947
:10337000624071058105910569F160F1A0903E06FA
:10338000B0903F06C0904006D0904106E0904206C3
:10339000F090430600914406109145062CA13EA1F1
:1033A00048A5552D6B2F7A2F8F2F9E2F0E948B3083
:1033B00089F010923E0610923F061092400610923D
:1033C0004106109242061092430610924406109253
:1033D000450624C1709026068091270689A3909106
:1033E00028069AA3109129061BA330902A06409024
:1033F0002B0660902C0620902D06CE010D964C01D8
:10340000A72CB9A0CAA0D12EE32CF42C062D122D86
:103410002CA13EA148A5552D6B2F7A2F8F2F9E2FC3
:103420000E942A0F61E070E082E090E00E94951413
:10343000512C38C07092260699A1909327061AA1A4
:10344000109328068BA18093290630922A06409279
:103450002B0660922C0620922D06CE010D964C0173
:10346000A12CB12CC12CD12CE12CF12C00E010E0CE
:103470002CA13EA148A5552D6B2F7A2F8F2F9E2F63
:103480000E942A0F722E39A34AA35BA3362E472E21
:10349000682E292E61E070E082E090E00E94951491
:1034A00055245394298D3A8D4B8D5C8D6D8D7E8D79
:1034B0008F8D98A130584A415640610971098109A0
:1034C00091092F37304E42475849624071058105B6
:1034D000910509F008F457C082E080934E062091D0
:1034E0003606309137064091380650913906609182
:1034F0003A0670913B0680913C0690913D06A0E013
:103500000E94943009F442C086E396E00E943C1188
:103510008BA7A0902606B0902706C0902806D090D2
:103520002906E0902A06F0902B0600912C061091B7
:103530002D0620913606309137064091380650917D
:10354000390660913A0670913B06CE0101964C0116
:1035500080913C0690913D060E942A0F1F928BA4F9
:10356000A12CC980DA80EB80FC800D811E812F8127
:10357000388549855A856B857C8581E090E00E947D
:10358000BA130F9003C088E080934E06898D809314
:103590003E068A8D80933F068B8D809340068C8DEE
:1035A000809341068D8D809342068E8D80934306D5
:1035B0008F8D8093440688A18093450681E090E03A
:1035C0009DA38CA302C01FA2512C9FA19F938BA4EB
:1035D000AFA0CD84DE84EF84F88809891A892B890D
:1035E0003C894D895E896F89788D89A59AA50E944D
:1035F000BA130F90E1E05E1210C00CA11DA1272D9F
:1036000039A14AA15BA1632D742D862D922D0E94B4
:10361000AE1403C09924939401C0912C892DAB96CC
:103620000FB6F894DEBF0FBECDBFDF91CF911F91D3
:103630000F91FF90EF90DF90CF90BF90AF909F9051
:103640008F907F906F905F904F903F902F90089554
:10365000CF93DF93EC0141E050E06CE473E00E9413
:103660004B0A811103C0CE010E94B20ACE01DF9144
:10367000CF910895E0915306F09154060190F081A6
:10368000E02D682F83E596E009948F929F92AF9288
:10369000BF920F931F93CF93DF93CDB7DEB7A19760
:1036A0000FB6F894DEBF0FBECDBF19A2423008F4AA
:1036B0004AE08E010F5D1F4F842E912CA12CB12C5E
:1036C000A50194010E94C82EE62FB901CA0101503C
:1036D0001109EA3014F4E05D01C0E95CD801EC9313
:1036E000232B242B252B61F7B80183E596E00E945C
:1036F000940BA1960FB6F894DEBF0FBECDBFDF913D
:10370000CF911F910F91BF90AF909F908F90089590
:103710004F925F926F927F928F929F92AF92BF92E1
:10372000CF92DF92EF92FF926B017C01B42E9B014E
:10373000AC010E949F2E882319F069ED73E027C029
:1037400026013701E89477F82FEF3FEF4FE75FE767
:10375000C301B2010E949F2E81110DC02FEF3FEFD8
:103760004FE75FE7C301B2010E94FA2B18161CF461
:103770006DED73E00CC02FEF3FEF4FE75FE4C70143
:10378000B6010E949A2E181694F461EE73E083E558
:1037900096E0FF90EF90DF90CF90BF90AF909F901A
:1037A0008F907F906F905F904F900C94940B2FEFC1
:1037B0003FEF4FE75FECC701B6010E94FA2B87FD90
:1037C000E4CF20E030E0A901C701B6010E94FA2B46
:1037D00087FF09C08DE20E943A1B4C01F7FAF09472
:1037E000F7F8F09402C0812C912CA12C60E070E0DD
:1037F00080E09FE3AB1441F020E030E040E251E490
:103800000E94F22DA394F6CF9B01AC01C701B60133
:103810000E94862D2B013C010E946B2E6B017C01C6
:103820000E94FF2B9B01AC01C301B2010E94852DB8
:103830002B013C014AE0C701B6010E94451B7C01F7
:10384000E80CF91CBB2029F08EE20E943A1BE80E1E
:10385000F91EDB2CDD2021F120E030E040E251E4D4
:10386000C301B2010E94602C2B013C010E946B2E0F
:103870004B01A12CB12C4AE0C501B4010E94451BAB
:10388000E80EF91EC501B4010E94FF2B9B01AC019B
:10389000C301B2010E94852D2B013C01DA94DACFDD
:1038A000C701FF90EF90DF90CF90BF90AF909F90B7
:1038B0008F907F906F905F904F900895CF93DF939C
:1038C000CDB7DEB728970FB6F894DEBF0FBECDBFD9
:1038D00028E0E3EBF1E0DE01119601900D922A95CC
:1038E000E1F720915C06261710F46FEF620FFE01DE
:1038F0003196E60FF11DE60FF11D9081682F690FDB
:10390000606840E083E596E028960FB6F894DEBF45
:103910000FBECDBFDF91CF910C945F0DCF92DF92A0
:10392000EF92FF92CF93DF9397FF19C06B017C0159
:103930008DE20E943A1BEC0166277727CB016C19B8
:103940007D098E099F094AE00E94451B8C0F9D1F2F
:10395000DF91CF91FF90EF90DF90CF9008954AE0F4
:10396000DF91CF91FF90EF90DF90CF900C94451BAB
:10397000CF93DF9300D0CDB7DEB789831A8241E0C1
:1039800050E0BE016F5F7F4F86E096E00E944B0AD9
:103990000F900F90DF91CF910895009769F0FC018F
:1039A00001900020E9F73197AF01481B590BBC018A
:1039B00084E995E00C944B0A80E00895CF93DF935F
:1039C000CDB7DEB7E2970FB6F894DEBF0FBECDBF1E
:1039D000789484B5826084BD84B5816084BD85B5EA
:1039E000826085BD85B5816085BD80916E008160F6
:1039F00080936E001092810080918100826080939C
:103A0000810080918100816080938100809180009D
:103A10008160809380008091B10084608093B100C8
:103A20008091B00081608093B00080917A008460C2
:103A300080937A0080917A00826080937A008091EE
:103A40007A00816080937A0080917A008068809308
:103A50007A001092C10010927B0410927A041092A6
:103A6000C4041092E6040E940C0F10925806809134
:103A70005C06823018F098E09093580690915D06AD
:103A8000992339F0813029F480915806846080931D
:103A9000580662E370E080E090E00E94AF0C609115
:103AA0005E0683E596E00E94330D68EE73E080E0E9
:103AB00090E00E94AF0C60E383E596E00E94460D23
:103AC0000BE416E4C8010197F1F760E383E596E0A3
:103AD0000E94460DC8010197F1F760E383E596E087
:103AE0000E94460D83E592E00197F1F760E283E5DD
:103AF00096E00E94460D60915806606240E083E5C2
:103B000096E00E945F0D84E08093590640E06CE0EF
:103B100083E596E00E945F0D40E061E083E596E07A
:103B20000E945F0D0BE31FE1C8010197F1F782E0EE
:103B300080935A0640E066E083E596E00E945F0DC0
:103B400040E062E083E596E00E945F0DC8010197C6
:103B5000F1F788E080935E0660E083E596E00E94DE
:103B6000330D80E090E00E941E2D8093FA03873F82
:103B700029F481E10E94030C892BA1F567EF698389
:103B80001A8280E090E06FA70E941E2D67EF6817F1
:103B900021F080E090E00E94262D6A8181E090E093
:103BA0006FA70E941E2D6FA5681721F081E090E09D
:103BB0000E94262D60E471E08AE090E00E94F60009
:103BC0006CE371E084E190E00E94F60060E975E04A
:103BD0008EE190E00E94F60068E371E088E290E0F8
:103BE0000E94F60068E371E088E290E00E94D00055
:103BF000FC0180819181A281B3818115914EA10543
:103C0000B105D1F5E091F704F091F80482E08083EA
:103C1000E091F704F091F8041082E091F304F09140
:103C2000F4041082E091F504F091F60480E18083C1
:103C30001092FF04E091FB04F091FC0486E0808385
:103C4000E091F904F091FA04808180618083E09131
:103C5000F904F091FA04808188608083E091F9048E
:103C6000F091FA04808180688083E091F904F091FA
:103C7000FA0480818F7D808368E371E088E290E0C0
:103C80000E94D000FC0180819181A281B3818115C5
:103C9000924CA140B105A9F5E091F704F091F80428
:103CA00082E08083E091F304F091F4041082E091CB
:103CB000F504F091F60480E180831092FF04E09116
:103CC000FB04F091FC0486E08083E091F904F0911C
:103CD000FA04808180618083E091F904F091FA0414
:103CE000808188608083E091F904F091FA048081FA
:103CF00080688083E091F904F091FA0480818F7DDF
:103D0000808361E084E00E945C0C60E085E00E94BA
:103D10005C0C61E086E00E945C0C61E087E00E9440
:103D20005C0C61E088E00E945C0C61E089E00E942C
:103D30005C0C61E08AE00E945C0C61E08BE00E9418
:103D40005C0C61E08CE00E945C0C61E08DE00E9404
:103D50005C0C60E080E10E945C0C60E081E10E940C
:103D60005C0C62E080E10E945C0C62E085E00E94F5
:103D70005C0C62E081E10E945C0C809168008460D0
:103D80008093680080916D008C6080936D007894C2
:103D900060E471E08AE090E00E94D000FC01808144
:103DA0009181A281B3818093400190934101A093BE
:103DB0004201B09343016CE371E084E190E00E9422
:103DC000D000FC0180819181A281B38180933C016C
:103DD00090933D01A0933E01B0933F0160E975E0EF
:103DE0008EE190E00E94D000DC016D917D918D917B
:103DF0009C916093900570939105809392059093A8
:103E0000930524E630E040E050E00E94682F2093C4
:103E10004D0130934E0140934F01509350016093F8
:103E200051017093520180935301909354018091FA
:103E3000400190914101A0914201B09143018093D2
:103E4000490690934A06A0934B06B0934C06C09047
:103E50003C01D0903D01E0903E01F0903F01109276
:103E60007B0410927A041092C4041092E6040E941B
:103E70000C0F62E987EB0E943A13C114D104E104EC
:103E8000F10409F44EC08FE00E945313682F6F7342
:103E9000B1E8CB16B3ECDB06B9ECEB06B1E0FB0600
:103EA00048F4C0924F06D0925006E0925106F0922C
:103EB000520634C0D701C6018158934CA94CB14079
:103EC0008038934CA94CB14070F4F694E794D794A1
:103ED000C794C0924F06D0925006E0925106F092DD
:103EE000520660641BC0D701C60181509748A349A0
:103EF000B34081159A45A246B24080F412E0F69490
:103F0000E794D794C7941A95D1F7C0924F06D092F0
:103F10005006E0925106F092520660688FE00E94CF
:103F20003A1360E880E10E943A1360E881E10E9460
:103F30003A1360E882E10E943A136CE080E10E944B
:103F40003A136CE081E10E943A136CE082E10E9436
:103F50003A1360E281EB0E943A1360E881EB0E9421
:103F60003A1320914D0130914E0140914F015091F3
:103F700050016091510170915201809153019091D3
:103F8000540100E010E00E94AE14A0904D01B090EA
:103F90004E01C0904F01D0905001E0905101F0903F
:103FA0005201009153011091540180914801909168
:103FB0004901A0914A01B0914B0188529342A10955
:103FC000B109BC01CD01B2E0660F771F881F991FB0
:103FD000BA95D1F724E630E040E050E00E94682F27
:103FE000812C912C0E94991680E10E9453138C7FA2
:103FF000682F626080E10E943A1360E371E081E023
:104000000E940B1368E271E082E00E940B1360E2F1
:1040100071E083E00E940B1368E171E084E00E948C
:104020000B1360E171E085E00E940B1368E071E022
:1040300086E00E940B1360E071E087E00E940B13A2
:104040008090F6039090F703A090F803B090F903E6
:1040500081149104A104B10409F492C0C0904401F8
:10406000D0904501E0904601F09047016091FB033C
:104070007091FC038091FD039091FE03A7019601CE
:104080000E94EA2E280D391D4A1D5B1DC701B6018D
:104090000E94A42E6093FB037093FC038093FD03A6
:1040A0009093FE031AA619A61CA61BA61EA61DA663
:1040B0002AE0AE014F5F5F4F0E948A2BBE016F5F07
:1040C0007F4FCE0189960E94F80A8DA59EA50B9779
:1040D00030F51CA21BA21EA21DA218A61FA24AE018
:1040E000BE016F5F7F4F80E090E00E947F2BBE019A
:1040F0006F5F7F4FCE0183960E94F80ABE01675D15
:104100007F4FCE0183960E94C40ABC01CE018996DE
:104110000E940F0BCE0183960E94260BD6CF6BEB2D
:1041200071E0CE0101960E942B0BBE01675D7F4FAF
:10413000CE0101960E94C40A0E94281BBC01CE0138
:1041400089960E940F0BCE0101960E94260BBE019C
:10415000675D7F4F87EE94E00E94860B60E570E01C
:1041600080E090E00E94AF0C1092F6031092F703EB
:104170001092F8031092F903CE0189960E94260B43
:104180000E94D0071CA21BA21EA21DA218A61FA23D
:1041900066E076E0CE0183960E940F0B2DE030E0C2
:1041A00042E050E0BE016D5D7F4FCE0101960E945E
:1041B000400BBE016F5F7F4F88EE95E00E94790A49
:1041C000CE0101960E94260B88EE95E00E94210AFE
:1041D000609348017093490180934A0190934B0189
:1041E0006093FB037093FC038093FD039093FE03A5
:1041F0002EE130E04DE150E0BE016D5D7F4FCE011C
:1042000001960E94400BBE016F5F7F4F82EE95E0EA
:104210000E94790ACE0101960E94260B82EE95E05B
:104220000E94210A613029F41092140469ED71E0B2
:1042300039C0623029F4609314046EEB71E032C02F
:10424000633031F484E08093140461EC71E02AC09F
:10425000643031F485E08093140464EC71E022C092
:10426000653031F486E08093140467EC71E01AC085
:10427000663031F489E0809314046AEC71E012C076
:10428000673031F483E0809314046DEC71E00AC070
:10429000693019F06093140409C087E08093140416
:1042A00060ED71E082EE95E00E94F80A21E230E0D4
:1042B00040E250E0BE016D5D7F4FCE0101960E944D
:1042C000400BBE016F5F7F4F8CE096E00E94790A41
:1042D000CE0101960E94260B8CE096E00E94210AF6
:1042E000062F60931A0428E130E047E150E0BE0158
:1042F0006D5D7F4FCE0101960E94400BBE016F5F46
:104300007F4F8AEF95E00E94790ACE0101960E94C4
:10431000260B8AEF95E00E94210A6093130429E19D
:1043200030E048E150E0BE016D5D7F4FCE01019667
:104330000E94400BBE016F5F7F4F84EF95E00E94AB
:10434000790ACE0101960E94260B84EF95E00E9427
:10435000210A6093120421E130E04DE050E0BE01FB
:104360006D5D7F4FCE0101960E94400BBE016F5FD5
:104370007F4F8CED95E00E94790ACE0101960E9454
:10438000260B22E130E041E150E0BE016D5D7F4F40
:10439000CE0101960E94400BBE016F5F7F4F80ED02
:1043A00095E00E94790ACE0101960E94260B27E132
:1043B00030E042E150E0BE016D5D7F4FCE010196DD
:1043C0000E94400BBE016F5F7F4F86ED95E00E941B
:1043D000790ACE0101960E94260B86ED95E00E9497
:1043E000210A60930E0470930F048093100490933D
:1043F00011042DE130E04CE150E0BE016D5D7F4FD6
:10440000CE0101960E94400BBE016F5F7F4F80E09E
:1044100096E00E94790ACE0101960E94260B80E068
:1044200096E00E94210A162F6093F50364E772E07C
:1044300086E096E00E94F80ACE0183960E94260B41
:10444000013009F086C0113009F083C063ED71E0DE
:1044500087EE94E00E94A90B87EE94E00E94480941
:1044600068E270E080E090E00E94AF0C87EE94E09C
:104470000E94CA08181619060CF05FC087EE94E077
:104480000E94A8088093E7038F3321F40E94AB02B7
:104490000E94AC058091E7038634A9F18091E60380
:1044A000882309F44AC066E076E080EA95E00E943D
:1044B0000F0B2DE030E044E050E060EA75E0CE0103
:1044C00001960E94400BBE016F5F7F4F8AE995E025
:1044D0000E94790ACE0101960E94260B8AE995E096
:1044E0000E94210A6093FF037093000480930104EB
:1044F00090930204609348017093490180934A01AC
:1045000090934B011AC086E40E94B81C01E087EE2C
:1045100094E00E94CA08181619060CF0BFCF87EE67
:1045200094E00E94A808182F8093E7030E94B81C0B
:104530001B3369F70093E603EACF64E772E080EA91
:1045400095E00E94F80A64E772E086E096E00E9437
:10455000F80A67ED71E08CED95E00E942C0A882343
:1045600029F081E090E0A0E0B0E0B5C06CED71E032
:104570008CED95E00E942C0A882329F08AE090E0D7
:10458000A0E0B0E0A8C061EE71E08CED95E00E9483
:104590002C0A882329F082E390E0A0E0B0E09BC0E1
:1045A00066EE71E08CED95E00E942C0A882329F0DC
:1045B00084E690E0A0E0B0E08EC06BEE71E08CEDA0
:1045C00095E00E942C0A882329F08AEF90E0A0E071
:1045D000B0E081C060EF71E08CED95E00E942C0AA4
:1045E000882329F084EF91E0A0E0B0E074C065EF8B
:1045F00071E08CED95E00E942C0A882329F088EE6A
:1046000093E0A0E0B0E067C06AEF71E08CED95E068
:104610000E942C0A882329F084EC99E0A0E0B0E005
:104620005AC06FEF71E08CED95E00E942C0A882350
:1046300029F088E893E1A0E0B0E04DC064E072E0CA
:104640008CED95E00E942C0A882329F08AE698E1F7
:10465000A0E0B0E040C069E072E08CED95E00E941F
:104660002C0A882329F088E293E2A0E0B0E033C06E
:104670006EE072E08CED95E00E942C0A882329F010
:1046800080E197E2A0E0B0E026C063E172E08CED4B
:1046900095E00E942C0A882329F084ED90E3A0E0A5
:1046A000B0E019C068E172E08CED95E00E942C0A40
:1046B000882329F088E99AE3A0E0B0E00CC06DE11E
:1046C00072E08CED95E00E942C0A882361F080E274
:1046D0009EE4A0E0B0E08093440190934501A09354
:1046E0004601B093470160E070E0CB010E94AF0C3F
:1046F0000E94DB020E94E9061091EF03113091F451
:1047000080910504813071F062E272E087EE94E0FE
:104710000E94A90B68E270E080E090E00E94AF0C7C
:10472000109305048091EF03811112C0809105045C
:10473000813071F466E272E087EE94E00E94A90B8A
:1047400068E270E080E090E00E94AF0C10920504F7
:104750008091F5038130B9F561E084E00E942C0C72
:1047600000910304109104040F5F1F4F1093040481
:104770000093030483E10E94980CBC01990F880BFD
:10478000990B0E94012C6B017C0186E10E94980C20
:10479000BC01990F880B990B0E94012C2B013C0145
:1047A0009B01AC01C701B6010E949A2E87FD12C081
:1047B00061E080E00E945E1C6AE272E083E596E0C0
:1047C0000E94A90BA3C08111A1C060E084E00E94F7
:1047D0002C0C9CC00115110521F0033011050CF4BF
:1047E00095C0A7019601C301B2010E94862D4B011D
:1047F0005C01A7019601C301B2010E94852D9B01B6
:10480000AC01C501B4010E94F22D6B017C0120E0D6
:1048100030E0A9010E949A2E181624F0F7FAF094BD
:10482000F7F8F09420E030E040EA50E4C301B20130
:104830000E94602C20E030EC4FE754E40E94F22DFF
:104840002CE238E540EB5CE30E94F22D9B01AC01C9
:104850000E94602C20E030E048E452E40E94F22DF7
:104860002B013C0120E030E040E050E4C701B601FC
:104870000E94862D4B015C01A701960160E070E06B
:1048800080E89FE30E94F22D9B01AC01C501B401B9
:104890000E94862D9B01AC0160E070E080E890E40E
:1048A0000E94F22D9B01AC01C301B2010E94602C59
:1048B0004B015C0161E080E00E945E1C6DE372E0F0
:1048C00083E596E00E94A90B42E0C701B6010E9471
:1048D000881B61E088E00E945E1C62E472E083E570
:1048E00096E00E94A90B61E08BE00E945E1C40E014
:1048F000C501B4010E94881B66E472E083E596E07E
:104900000E94A90B10920404109203048091F403F6
:104910008F5F8093F4038A3041F48091F5038130F6
:1049200021F01092F4030E9434068091F0039091DC
:10493000F103892B09F0B3C160E083E00E945E1CA3
:10494000609148017091490180914A0190914B0119
:1049500020E432E44FE050E00E94EA2E2A30310594
:1049600058F480E22FA738AB49AB5AAB0E943A1BF0
:104970005AA949A938A92FA5CA01B9018827992799
:104980004AE00E94451B8EE20E943A1B609148015A
:104990007091490180914A0190914B0120E432E4E9
:1049A0004FE050E00E94EA2E28EE33E040E050E075
:1049B0000E94EA2E890124363105A8F480E32FA74E
:1049C00038AB49AB5AAB0E943A1B2FA538A949A96D
:1049D0005AA90A30110538F480E30E943A1B5AA9FB
:1049E00049A938A92FA5CA01B901882799274AE002
:1049F0000E94451B8EE20E943A1B60914801709113
:104A0000490180914A0190914B0128EE33E040E04A
:104A100050E00E94EA2E6B017C018B016436710527
:104A200048F480E30E943A1B0A30110518F480E331
:104A30000E943A1BC701B601882799274AE00E94C5
:104A4000451B60E08DE00E945E1C63E373E083E53C
:104A500096E00E94A90B8091F203813049F1809188
:104A6000EF0381110DC08091F503811109C060E051
:104A70000E945E1C6BE472E083E596E00E94A90B45
:104A80008091EF03813021F08091F503813081F432
:104A900064E872E083E596E00E94A90B60E080E0A4
:104AA0000E945E1C6FE472E083E596E00E94A90B11
:104AB0008091F203813051F460E080E00E945E1C3E
:104AC00063E572E083E596E00E94A90B8091F5030F
:104AD0008111F1C08091EE03811109C061E00E9453
:104AE0005E1C67E572E083E596E00E94A90B809169
:104AF000EE03813051F461E080E00E945E1C6CE5C1
:104B000072E083E596E00E94A90B8091EE0382306B
:104B100051F461E080E00E945E1C61E672E083E592
:104B200096E00E94A90B8091EE03833051F461E07E
:104B300080E00E945E1C66E672E083E596E00E94DB
:104B4000A90B2FB7F8948091E8039091E903A09105
:104B5000EA03B091EB032FBF40910A0450910B047C
:104B600060910C0470910D04841B950BA60BB70B80
:104B7000853F9140A105B10508F49DC00E94AC0598
:104B800064E772E084E995E00E94F80A8091EC0302
:104B90009091ED038C3891050CF094C344976CE030
:104BA00070E00E94B42E161617060CF486C31092FD
:104BB0000904109208048091080490910904893036
:104BC0009105E4F08BE692E00E94CD1C61E08DE05F
:104BD0000E945E1C65E772E083E596E00E94A90BE7
:104BE0006091060470910704072E000C880B990B46
:104BF0000E948E1C80E20E943A1B33C088309105CF
:104C000019F487E792E02BC08730910519F487E803
:104C100092E025C08630910519F487E992E01FC023
:104C20008530910519F487EA92E019C08430910526
:104C300019F487EB92E013C08330910519F487ECE7
:104C400092E00DC08230910519F487ED92E007C023
:104C5000019719F487EE92E002C087EF92E00E947C
:104C6000CD1C61E084E00E945E1C64E975E083E590
:104C700096E00E94860B2FB7F8948091E8039091FC
:104C8000E903A091EA03B091EB032FBF80930A04DC
:104C900090930B04A0930C04B0930D040CC00E94DD
:104CA000A0038091F0039091F103059724F01092F6
:104CB000F1031092F0038091480190914901A09175
:104CC0004A01B0914B01813A9648A140B10564F484
:104CD00080EA96E8A1E0B0E0809348019093490112
:104CE000A0934A01B0934B018091480190914901F2
:104CF000A0914A01B0914B01803C9540A94DB14033
:104D000084F08091F303813061F080EC95E0A9EDAF
:104D1000B1E08093480190934901A0934A01B09378
:104D20004B01909114048091F5039530B9F48130D2
:104D3000A9F48091480190914901A0914A01B09154
:104D40004B01885F9A42A109B10980934801909371
:104D50004901A0934A01B0934B0123C081111EC0A9
:104D600080911304811105C0809112048111C6C283
:104D700008C0813009F066C080911204813009F0CA
:104D8000C1C28091480190914901A0914A01B0911E
:104D90004B0188529342A109B1094CC0813009F0FE
:104DA00051C08091130481114DC080911204813053
:104DB00009F048C065E772E080ED95E00E942C0A9A
:104DC0008823E1F0409148015091490160914A01E6
:104DD00070914B0180910E0490910F04A0911004EA
:104DE000B0911104840F951FA61FB71F809348012F
:104DF00090934901A0934A01B0934B0169E073E09D
:104E000080ED95E00E942C0A8823E1F08091480112
:104E100090914901A0914A01B0914B0140910E043B
:104E200050910F046091100470911104841B950B34
:104E3000A60BB70B8093480190934901A0934A01B8
:104E4000B0934B01809119048F5F8F3019F08093DC
:104E5000190402C010921904409048015090490171
:104E600060904A0170904B01809115049091160456
:104E7000A0911704B0911804481659066A067B06DB
:104E800009F462C1A0904D01B0904E01C0904F0155
:104E9000D0905001E0905101F090520100915301E7
:104EA00010915401C301B201A2E0660F771F881F61
:104EB000991FAA95D1F724E630E040E050E00E9427
:104EC000682F812C912C0E949916D301C201805425
:104ED0009244AF40B10980389448AE41B105B8F46E
:104EE00061E08CE00E942C0C60E08BE00E942C0CB6
:104EF00060E08AE00E942C0C60E089E00E942C0CAB
:104F000060E088E00E942C0C6BE073E00CC1D301E0
:104F1000C201805C964CAD42B10980389448AE41E4
:104F2000B105B8F460E08CE00E942C0C61E08BE0ED
:104F30000E942C0C60E08AE00E942C0C60E089E06A
:104F40000E942C0C60E088E00E942C0C6FE073E063
:104F5000EAC0D301C20180549B44AC44B109803CF7
:104F6000964CAD42B105B8F460E08CE00E942C0C88
:104F700060E08BE00E942C0C61E08AE00E942C0C27
:104F800060E089E00E942C0C60E088E00E942C0C1C
:104F900062E173E0C8C0D301C2019251AA47B109CE
:104FA00081159940AD43B105B8F460E08CE00E94F2
:104FB0002C0C60E08BE00E942C0C60E08AE00E94E8
:104FC0002C0C61E089E00E942C0C60E088E00E94DB
:104FD0002C0C65E173E0A7C0D301C2019B51A74B24
:104FE000B10981159940AD43B105B8F460E08CE09A
:104FF0000E942C0C60E08BE00E942C0C60E08AE0A8
:105000000E942C0C61E089E00E942C0C60E088E09A
:105010000E942C0C68E173E086C0D301C201945257
:10502000A44FB109803C964CAD42B105B8F460E0A4
:105030008CE00E942C0C60E08BE00E942C0C60E065
:105040008AE00E942C0C60E089E00E942C0C61E058
:1050500088E00E942C0C6BE173E065C0D301C201B3
:10506000805C9A4EA142B140803C964CAD42B10565
:10507000B8F460E08CE00E942C0C60E08BE00E94B1
:105080002C0C60E08AE00E942C0C60E089E00E9419
:105090002C0C61E088E00E942C0C6EE173E043C0B0
:1050A000D301C2018058914BAF44B14080349B443E
:1050B000AC44B105B8F460E08CE00E942C0C60E0D8
:1050C0008BE00E942C0C60E08AE00E942C0C60E0D7
:1050D00089E00E942C0C61E088E00E942C0C61E2C7
:1050E00073E021C0D301C201805C9C4FAB49B14049
:1050F00080349D45A64CB105D0F460E08CE00E9460
:105100002C0C60E08BE00E942C0C60E08AE00E9496
:105110002C0C60E089E00E942C0C61E088E00E9489
:105120002C0C68EE71E08EEB95E00E94F80A60E0CE
:1051300070E0CB010E94AF0C40921504509216040F
:1051400060921704709218042091C2053091C30533
:105150008091C8059091C9052817390739F58091C4
:10516000BE059091BF056091C4057091C50500977B
:1051700019F061157105B1F46115710551F0232B1A
:1051800009F449C0DB018C9190E0919581959109DA
:105190000BC0009709F43FC0232BE9F1FC0180818B
:1051A00090E002C00E94B932892BA9F180911A04C3
:1051B000811131C083E00E945313682F6D7F83E01B
:1051C0000E943A13A0904D01B0904E01C0904F0143
:1051D000D0905001E0905101F090520100915301A4
:1051E00010915401C301B201685B7E488F4F9F4FFD
:1051F00024E630E040E050E00E94682F8824839449
:10520000912C0E9499166EEB75E084EC95E00E945B
:105210000F0B10921904809119048E3041F483E031
:105220000E945313682F626083E00E943A138091BA
:10523000F303813081F53090F203F1E03F122BC08F
:1052400083E00E945313682F6B7F83E00E943A1320
:10525000A0904D01B0904E01C0904F01D0905001F0
:10526000E0905101F09052010091530110915401CE
:10527000C301B201685D7C4D8F4F9F4F24E630E043
:1052800040E050E00E94682FE2E08E2E912C0E94B8
:1052900099163092F2038091F20381110AC083E0E3
:1052A0000E945313682F646083E00E943A131092A7
:1052B000F3030E946A090C94202070930904609300
:1052C000080479CC29E030E03093090420930804E5
:1052D000BC0166587109072E000C880B990B0E94BF
:1052E000012C2FE832EC45EF5EE30E94602C0E9417
:1052F000642E70930704609306045DCC813009F03E
:10530000A1CD3FCD81119ECDC0904801D0904901E3
:10531000E0904A01F0904B0188E2C81A83E2D80A73
:10532000E108F108C0924801D0924901E0924A0197
:10533000F0924B0165E772E080ED95E00E942C0A47
:10534000882309F45BCD80910E0490910F04A09105
:105350001004B0911104C80ED91EEA1EFB1EC092A3
:105360004801D0924901E0924A01F0924B0146CDAA
:1053700084E995E00E94260B8AE995E00E94260BBD
:1053800080EA95E00E94260B86EA95E00E94260BB3
:105390008CEA95E00E94260B82EB95E00E94260B9A
:1053A00088EB95E00E94260B8EEB95E00E94260B81
:1053B00084EC95E00E94260B8AEC95E00E94260B77
:1053C00080ED95E00E94260B86ED95E00E94260B6D
:1053D0008CED95E00E94260B82EE95E00E94260B54
:1053E00088EE95E00E94260B8EEE95E00E94260B3B
:1053F00084EF95E00E94260B8AEF95E00E94260B31
:1054000080E096E00E94260B86E096E00E94260B44
:105410008CE096E00C94260BAF92BF92CF92DF9275
:10542000EF92FF920F931F93CF93DF93E7EEF4E099
:105430001382128288EE93E0A0E0B0E0848395832B
:10544000A683B7832BE731E03183208325EC30E05E
:105450003587248724EC30E03787268720EC30E03E
:10546000318B208B21EC30E0338B228B22EC30E02F
:10547000358B248B26EC30E0378B268B118E128EE9
:10548000138E148EE4E8F5E01382128284839583F0
:10549000A683B7838DE891E091838083E3E5F6E00E
:1054A000138212828FE991E09183808387E2848363
:1054B00080E1808792E09187128688E08387E5E12A
:1054C000F6E080AF81AF11AA12AA13AA1186128644
:1054D00013861486158616861786108A118A128AF4
:1054E000138A148A158A168A178A108E118E128EC4
:1054F000138E148E158E168E178E10A211A212A264
:1055000013A214A215A216A217A210A611A612A6E3
:1055100013A614A615A616A617A610AA40EC5CEFB3
:105520006BE971E042AF53AF64AF75AFC2E1D6E053
:10553000998383E08A8360E082E00E945C0C60E0F3
:105540008A810E945C0C61E089810E942C0C61E0E0
:105550008A810E942C0C188264E772E08CE096E04D
:105560000E942B0B64E772E086E096E00E942B0B12
:1055700064E772E080E096E00E942B0B64E772E043
:105580008AEF95E00E942B0B64E772E084EF95E0D0
:105590000E942B0B64E772E08EEE95E00E942B0BCD
:1055A00064E772E088EE95E00E942B0B64E772E0FE
:1055B00082EE95E00E942B0B64E772E08CED95E0A3
:1055C0000E942B0B64E772E086ED95E00E942B0BA6
:1055D00064E772E080ED95E00E942B0B64E772E0D7
:1055E0008AEC95E00E942B0B64E772E084EC95E076
:1055F0000E942B0B64E772E08EEB95E00E942B0B70
:1056000064E772E088EB95E00E942B0B64E772E0A0
:1056100082EB95E00E942B0B64E772E08CEA95E048
:105620000E942B0B64E772E086EA95E00E942B0B48
:1056300064E772E080EA95E00E942B0B64E772E079
:105640008AE995E00E942B0B64E772E084E995E01B
:105650000E942B0B20914D0130914E0140914F0142
:10566000509150016091510170915201809153010C
:1056700090915401E4E6AE2EB12CC12CD12CE12C3A
:10568000F12C00E010E00E94D52F2093900530937C
:1056900091054093920550939305DF91CF911F910F
:1056A0000F91FF90EF90DF90CF90BF90AF90089553
:1056B0001F93FC0199278827BC01E89411911032AF
:1056C000E9F3193010F01E30C8F31B3251F01D32CF
:1056D00049F4689406C00E94992B610F711D811DC9
:1056E000911D119110531A30B0F33EF490958095AE
:1056F000709561957F4F8F4F9F4F1F910895BB27E6
:105700004A3031F4992322F4BDE2909581959F4F60
:105710000C94D12BBB272A3051F4992342F4BDE2DB
:1057200090958095709561957F4F8F4F9F4F0C940A
:10573000AF2B592F482F372F262F660F771F881F23
:10574000991F660F771F881F991F620F731F841F91
:10575000951F660F771F881F991F0895BB27FA01B1
:10576000A62F6217710581059105330B30FB66F09A
:10577000AA27660F771F881F991FAA1FA21710F06C
:10578000A21B63953850A9F7A05DAA3308F0A95D64
:10579000A19336F7B111B1931082CA010C94EA2B90
:1057A000BB27FB015527AA27880F991FAA1FA417FB
:1057B00010F0A41B83955051B9F7A05DAA3308F0EF
:1057C000A95DA193009779F7B111B1931192CB0123
:1057D0000C94EA2BDC01FC01672F71917723E1F730
:1057E000329704C07C916D9370836291AE17BF07AE
:1057F000C8F308950E943C2C08F481E00895E894D1
:1058000009C097FB3EF490958095709561957F4F08
:105810008F4F9F4F9923A9F0F92F96E9BB279395B6
:10582000F695879577956795B795F111F8CFFAF4C6
:10583000BB0F11F460FF1BC06F5F7F4F8F4F9F4FF7
:1058400016C0882311F096E911C0772321F09EE855
:10585000872F762F05C0662371F096E8862F70E0BB
:1058600060E02AF09A95660F771F881FDAF7880F95
:105870009695879597F90895990F0008550FAA0BEB
:10588000E0E8FEEF16161706E807F907C0F0121653
:105890001306E407F50798F0621B730B840B950B56
:1058A00039F40A2661F0232B242B252B21F40895AB
:1058B0000A2609F4A140A6958FEF811D811D089548
:1058C0000E94732C0C94E42C0E94D62C38F00E9479
:1058D000DD2C20F0952311F00C94CD2C0C94D32CBE
:1058E00011240C94182D0E94F52C70F3959FC1F390
:1058F000950F50E0551F629FF001729FBB27F00D7E
:10590000B11D639FAA27F00DB11DAA1F649F6627D2
:10591000B00DA11D661F829F2227B00DA11D621F21
:10592000739FB00DA11D621F839FA00D611D221FDB
:10593000749F3327A00D611D231F849F600D211DBF
:10594000822F762F6A2F11249F5750409AF0F1F042
:1059500088234AF0EE0FFF1FBB1F661F771F881FAB
:1059600091505040A9F79E3F510580F00C94CD2CEA
:105970000C94182D5F3FE4F3983ED4F38695779509
:105980006795B795F795E7959F5FC1F7FE2B880F51
:10599000911D9695879597F9089597F99F6780E8E7
:1059A00070E060E008959FEF80EC089500240A9471
:1059B0001616170618060906089500240A941216EA
:1059C0001306140605060895092E0394000C11F41D
:1059D000882352F0BB0F40F4BF2B11F460FF04C0CA
:1059E0006F5F7F4F8F4F9F4F089557FD9058440F23
:1059F000551F59F05F3F71F04795880F97FB991F2E
:105A000061F09F3F79F087950895121613061406EA
:105A1000551FF2CF4695F1DF08C016161706180677
:105A2000991FF1CF86957105610508940895E89452
:105A3000BB2766277727CB0197F90895F999FECF01
:105A400092BD81BDF89A992780B50895262FF999BE
:105A5000FECF1FBA92BD81BD20BD0FB6F894FA9A51
:105A6000F99A0FBE019608950E94762DA59F900D7C
:105A7000B49F900DA49F800D911D112408952F9225
:105A80003F924F925F926F927F928F929F92AF92CE
:105A9000BF92CF92DF92EF92FF920F931F93CF931B
:105AA000DF93CDB7DEB7CA1BDB0B0FB6F894DEBFB2
:105AB0000FBECDBF09942A88398848885F846E84D8
:105AC0007D848C849B84AA84B984C884DF80EE8022
:105AD000FD800C811B81AA81B981CE0FD11D0FB62B
:105AE000F894DEBF0FBECDBFED010895A29FB001B7
:105AF000B39FC001A39F700D811D1124911DB29F02
:105B0000700D811D1124911D08955058BB27AA279F
:105B10000E949D2D0C94E42C0E94D62C38F00E94FB
:105B2000DD2C20F039F49F3F19F426F40C94D32C8B
:105B30000EF4E095E7FB0C94CD2CE92F0E94F52C98
:105B400058F3BA17620773078407950720F079F4B2
:105B5000A6F50C94172D0EF4E0950B2EBA2FA02D60
:105B60000B01B90190010C01CA01A0011124FF270A
:105B7000591B99F0593F50F4503E68F11A16F04005
:105B8000A22F232F342F4427585FF3CF4695379504
:105B90002795A795F0405395C9F77EF41F16BA0BC9
:105BA000620B730B840BBAF09150A1F0FF0FBB1F77
:105BB000661F771F881FC2F70EC0BA0F621F731FC0
:105BC000841F48F4879577956795B795F7959E3F1D
:105BD00008F0B0CF9395880F08F09927EE0F9795AE
:105BE000879508950E94062E0C94E42C0E94DD2CCB
:105BF00058F00E94D62C40F029F45F3F29F00C9415
:105C0000CD2C51110C94182D0C94D32C0E94F52CF2
:105C100068F39923B1F3552391F3951B550BBB27DB
:105C2000AA2762177307840738F09F5F5F4F220F20
:105C3000331F441FAA1FA9F335D00E2E3AF0E0E817
:105C400032D091505040E695001CCAF72BD0FE2F61
:105C500029D0660F771F881FBB1F261737074807F5
:105C6000AB07B0E809F0BB0B802DBF01FF279358AD
:105C70005F4F3AF09E3F510578F00C94CD2C0C9478
:105C8000182D5F3FE4F3983ED4F38695779567959A
:105C9000B795F7959F5FC9F7880F911D96958795E2
:105CA00097F90895E1E0660F771F881FBB1F621701
:105CB00073078407BA0720F0621B730B840BBA0BBF
:105CC000EE1F88F7E09508950E946B2E6894B1113D
:105CD0000C94182D08950E94FD2C88F09F5798F081
:105CE000B92F9927B751B0F0E1F0660F771F881FE1
:105CF000991F1AF0BA95C9F714C0B13091F00E94FB
:105D0000172DB1E008950C94172D672F782F882751
:105D1000B85F39F0B93FCCF3869577956795B39521
:105D2000D9F73EF490958095709561957F4F8F4F90
:105D30009F4F08950E943C2C08F48FEF08950E9415
:105D40003C2C880B990B0895DB018F939F930E9445
:105D5000342DBF91AF91A29F800D911DA39F900DF7
:105D6000B29F900D1124089597FB072E16F400940E
:105D700007D077FD09D00E94A03007FC05D03EF483
:105D8000909581959F4F0895709561957F4F0895E7
:105D9000A1E21A2EAA1BBB1BFD010DC0AA1FBB1F2F
:105DA000EE1FFF1FA217B307E407F50720F0A21BA1
:105DB000B30BE40BF50B661F771F881F991F1A940E
:105DC00069F760957095809590959B01AC01BD0138
:105DD000CF010895052E97FB1EF400940E94012F19
:105DE00057FD07D00E94C82E07FC03D04EF40C9438
:105DF000012F50954095309521953F4F4F4F5F4F64
:105E0000089590958095709561957F4F8F4F9F4F26
:105E10000895EE0FFF1F0590F491E02D0994DF9394
:105E2000CF931F930F939A9DF02D219FF00D8B9D83
:105E3000F00D8A9DE02DF10D039FF00D029FE00D06
:105E4000F11D4E9DE00DF11D5E9DF00D4F9DF00D7D
:105E50007F936F93BF92AF925F934F93D5010E9450
:105E6000762D8B01AC01D7010E94762DEB01E80F56
:105E7000F91FD6010E945F2F2F913F91D6010E94FA
:105E8000762DC60FD71FE81FF91FAF91BF910E9453
:105E90005F2F2F913F910E94762DC60FD71FE81FCD
:105EA000F91FD6010E94762DE60FF71F9801BE015B
:105EB000CF0111240F911F91CF91DF9108950E947E
:105EC000762D460F571FC81FD91F08F43196089525
:105ED00097FB57FF0C94782F9F938F930E94782FF6
:105EE0006E1B7F0BAF91BF918A0B9B0B0895E894BB
:105EF000DF93CF93FC01DB010E94762D7F936F939C
:105F0000E9019A01AC01BF93AF933F932F93DF0157
:105F10000E94762D26F46C1B7D0B820B930B9E0149
:105F2000EB01FC010E945F2FAF91BF912F913F9138
:105F30000E945F2FBE01CF01F9012F913F91CF91B8
:105F4000DF910895689401C0E894F92FF12B12F0C5
:105F50000C94D62FA0E0B0E0E0EBFFE20C94452DCE
:105F6000092E059422F40E943230112392F4F0E8B5
:105F70000F26FFEFE094F09400951095B094C09434
:105F8000D094A194BF0ACF0ADF0AEF0AFF0A0F0BD1
:105F90001F0B0E94E12F07FC0E943230CDB7DEB705
:105FA000ECE00C94612D689401C0E8948F929F926C
:105FB000CF93DF930E94E12FDF91CF919F908F903D
:105FC000089588249924F401E401B0E49F93AA275A
:105FD0009A158B049C04ED05FE05CF05D007A1079B
:105FE00098F4AD2FDC2FCF2FFE2FE92D982C892E82
:105FF000982F872F762F652F542F432F322F22274C
:10600000B85031F7BF9127C01B2EBF91BB27220F7D
:10601000331F441F551F661F771F881F991F881C39
:10602000991CEE1FFF1FCC1FDD1FAA1FBB1F8A1468
:106030009B04EC05FD05CE05DF05A007B10748F080
:106040008A189B08EC09FD09CE09DF09A00BB10BEA
:1060500021601A94E1F62EF49401AF01BE01CD0146
:10606000000C0895609570958095909530954095B9
:10607000509521953F4F4F4F5F4F6F4F7F4F8F4F41
:106080009F4F08950F93083090F0982F872F762F09
:10609000652F542F432F322F22270850F4CF220F81
:1060A000331F441F551F661F771F881F991F0A95AE
:1060B000B2F70F91089597FB10F8169400080F930C
:1060C000083098F00850232F342F452F562F672F74
:1060D000782F892F902DF4CF0594979587957795F4
:1060E000679557954795379527950A95AAF70F9184
:1060F00008952A0D3B1D4C1D5D1D6E1D7F1D801FCB
:10610000911F08952A193B094C095D096E097F0901
:10611000800B910B08952A153B054C055D056E0516
:106120007F058007910708950024A7FD00942A1792
:1061300030054005500560057005800590050895FF
:10614000AA1BBB1B51E107C0AA1FBB1FA617B7079D
:1061500010F0A61BB70B881F991F5A95A9F78095B9
:106160009095BC01CD010895CF93DF9382309105C6
:1061700010F482E090E0E0916106F091620620E088
:1061800030E0C0E0D0E0309711F1408151814817F4
:106190005907C0F04817590761F48281938120970D
:1061A00019F09B838A832BC09093620680936106CB
:1061B00026C02115310519F04217530718F49A012A
:1061C000BE01DF01EF010280F381E02DDCCF21155C
:1061D000310509F1281B390B2430310590F4129652
:1061E0008D919C9113976115710521F0FB019383AB
:1061F000828304C09093620680936106FD0132960B
:1062000044C0FD01E20FF31F8193919322503109A5
:106210002D933C933AC020915F0630916006232B6A
:1062200041F420915701309158013093600620933A
:106230005F0620915501309156012115310541F439
:106240002DB73EB74091590150915A01241B350B8F
:10625000E0915F06F0916006E217F307A0F42E1BB1
:106260003F0B2817390778F0AC014E5F5F4F2417BA
:10627000350748F04E0F5F1F5093600640935F064E
:106280008193919302C0E0E0F0E0CF01DF91CF91E4
:1062900008950F931F93CF93DF93009709F48CC059
:1062A000FC013297138212820091610610916206FE
:1062B0000115110581F420813181820F931F2091F6
:1062C0005F06309160062817390779F5F09360066C
:1062D000E0935F0671C0D80140E050E0AE17BF0701
:1062E00050F412962D913C911397AD012115310573
:1062F00009F1D901F3CF9D01DA0133832283608153
:106300007181860F971F8217930769F4EC0128812A
:106310003981260F371F2E5F3F4F318320838A81BB
:106320009B8193838283452B29F4F0936206E0934B
:10633000610642C01396FC93EE931297ED014991CA
:1063400059919E01240F351FE217F30771F48081E4
:106350009181840F951F029611969C938E93828152
:10636000938113969C938E931297E0E0F0E0D8010E
:1063700012968D919C911397009719F0F8018C015A
:10638000F6CF8D919C9198012E5F3F4F820F931F06
:1063900020915F06309160062817390769F430971D
:1063A00029F4109262061092610602C013821282D2
:1063B0001093600600935F06DF91CF911F910F91BC
:1063C0000895A0E0B0E0E7EEF1E30C94432DEC017A
:1063D000009721F4CB010E94B430B8C0FC01E60F55
:1063E000F71F9C0122503109E217F30708F4ACC0F3
:1063F000D9010D911C91119706171707B0F00530C0
:10640000110508F49FC0C80104978617970708F480
:1064100099C002501109061B170B019311936D933C
:106420007C93CF010E9449318DC05B01A01AB10A53
:106430004C01800E911EA0916106B091620640E071
:1064400050E0E12CF12C109709F44AC0A815B905C9
:10645000D1F56D907C901197630182E0C80ED11C3C
:10646000CA14DB0480F1A3014A195B096A0182E0C6
:10647000C80ED11C1296BC9012971396AC91B5E041
:10648000CB16D10440F0B282A38351834083D9015B
:106490006D937C930AC00E5F1F4FC301800F911F45
:1064A000F90191838083EB2DFA2FE114F10431F08F
:1064B000D7011396FC93EE93129744C0F0936206B3
:1064C000E09361063FC08D919C9111974817590741
:1064D00008F4AC017D0112960D90BC91A02DB3CFB4
:1064E00080915F069091600688159905E1F4461742
:1064F0005707C8F48091550190915601009741F4D7
:106500008DB79EB74091590150915A01841B950B4C
:10651000E817F907C8F4F0936006E0935F06F90105
:10652000718360830FC0CB010E94B4307C0100975F
:1065300059F0A801BE010E94B032CE010E9449313B
:10654000C70104C0CE0102C080E090E0CDB7DEB745
:10655000EEE00C945F2D81E090E0F8940C94C93249
:10656000FB01DC0102C001900D9241505040D8F770
:106570000895FB01DC018D91019080190110D9F380
:10658000990B0895FB01DC0101900D920020E1F7C9
:10659000089510E0C2E7D0E004C0FE010E94092F78
:0C65A0002196C337D107C9F7F894FFCF4C
:1065AC001F1115111D1D111F1F1115111515111F6F
:1065BC001F111D1D1D1D1D1F1F1117111515111F3D
:1065CC001F1117111D1D111F1F1515111D1D1D1F2D
:1065DC001F111D111D1D111F00E10000C0FC9B01AE
:1065EC00E86E030064000000A03B4C000100046B4B
:1065FC00F414000000000063068000000204000395
:10660C000001100302000003020100060004000652
:10661C00050020060504000000000001096E089921
:10662C00084809CA08A808BC0800000000A100DC42
:10663C000E9E00CC09F009DC09CD09000000008099
:10664C000D6E089E009D0000000000F8096E089E6B
:10665C00009D000000400014005400464100303200
:10666C000030340030350030360030390030330023
:10667C0030370046423B0030303030003030303163
:10668C0000313030300030303130003130303100BA
:10669C003130313000303031310031303131003176
:1066AC003130300030313030003031303100313168
:1066BC003031003131313000303131300030313156
:1066CC00310054583B0052583B0053575220202065
:1066DC00202020503D30572020202020005357529E
:1066EC003D0020503D0057202020005258200054DF
:1066FC0058200056464F004F666620004C6F77209E
:10670C00004D656420004869676800FFFFFFFFFFCC
:10671C00FFFFFF07002B00FFFFFFFFFFFFFF06201F
:10672C0020202020202000FFFFFFFFFFFF0520205E
:10673C0020202020202000FFFFFFFFFF042020202E
:10674C0020202020202000FFFFFFFF0320202020FE
:10675C0020202020202000FFFFFF022020202020CE
:10676C0020202020202000FFFF012020202020209E
:10677C0020202020202000FFFF202020202020206F
:10678C0020202020202000FF20202020202020203E
:10679C00202020202020002020202020202020200D
:1067AC002020202020202020002D003136300038E1
:1067BC0030003430003330003230003137003135A6
:1067CC000031320021002031392E3934382E30304E
:1067DC0030204D487A2000436F7252656620004687
:1067EC004130303030343939363030303B005A5A41
:1067FC004D4430323B00436F7272465245512E204D
:10680C0051554152545A0020487A0020436F7272FD
:10681C002E504C4C5F46495845442000434F4D2068
:10682C00504F52542052532D32333220005A5A4D6D
:10683C0044005A5A534D303B005A5A50413B005A6F
:10684C005A53443B005A5A53553B0042553B004265
:10685C00443B0049463B0020204E6F20636F6E6E18
:10686C00656374696F6E200020202020506F77655F
:10687C007253445220202020006E616E00696E66B7
:06688C00006F76660000BB
:00000001FF
